
D:\STM32\Program\1.11_Odchudzanie\um0427\FWLib\project\RIDE\STM3210E-EVAL\stm32f10x_tim.o:     file format elf32-littlearm
D:\STM32\Program\1.11_Odchudzanie\um0427\FWLib\project\RIDE\STM3210E-EVAL\stm32f10x_tim.o

Disassembly of section .text.TIM_TimeBaseInit:

00000000 <TIM_TimeBaseInit>:
TIM_TimeBaseInit():
D:\STM32\Program\1.11_Odchudzanie\um0427\FWLib\library\src/stm32f10x_tim.c:206
   0:	8803      	ldrh	r3, [r0, #0]
D:\STM32\Program\1.11_Odchudzanie\um0427\FWLib\library\src/stm32f10x_tim.c:199
   2:	b082      	sub	sp, #8
D:\STM32\Program\1.11_Odchudzanie\um0427\FWLib\library\src/stm32f10x_tim.c:206
   4:	f003 038f 	and.w	r3, r3, #143	; 0x8f
   8:	8003      	strh	r3, [r0, #0]
D:\STM32\Program\1.11_Odchudzanie\um0427\FWLib\library\src/stm32f10x_tim.c:207
   a:	8803      	ldrh	r3, [r0, #0]
   c:	88ca      	ldrh	r2, [r1, #6]
   e:	b29b      	uxth	r3, r3
  10:	4313      	orrs	r3, r2
  12:	884a      	ldrh	r2, [r1, #2]
  14:	4313      	orrs	r3, r2
  16:	b29b      	uxth	r3, r3
  18:	8003      	strh	r3, [r0, #0]
D:\STM32\Program\1.11_Odchudzanie\um0427\FWLib\library\src/stm32f10x_tim.c:210
  1a:	888b      	ldrh	r3, [r1, #4]
D:\STM32\Program\1.11_Odchudzanie\um0427\FWLib\library\src/stm32f10x_tim.c:199
  1c:	9001      	str	r0, [sp, #4]
D:\STM32\Program\1.11_Odchudzanie\um0427\FWLib\library\src/stm32f10x_tim.c:210
  1e:	8583      	strh	r3, [r0, #44]
D:\STM32\Program\1.11_Odchudzanie\um0427\FWLib\library\src/stm32f10x_tim.c:213
  20:	880b      	ldrh	r3, [r1, #0]
  22:	8503      	strh	r3, [r0, #40]
D:\STM32\Program\1.11_Odchudzanie\um0427\FWLib\library\src/stm32f10x_tim.c:216
  24:	f04f 0301 	mov.w	r3, #1	; 0x1
  28:	8283      	strh	r3, [r0, #20]
D:\STM32\Program\1.11_Odchudzanie\um0427\FWLib\library\src/stm32f10x_tim.c:218
  2a:	4b05      	ldr	r3, [pc, #20]	(40 <TIM_TimeBaseInit+0x40>)
  2c:	4298      	cmp	r0, r3
  2e:	d003      	beq.n	38 <TIM_TimeBaseInit+0x38>
  30:	f503 6300 	add.w	r3, r3, #2048	; 0x800
  34:	4298      	cmp	r0, r3
  36:	d101      	bne.n	3c <TIM_TimeBaseInit+0x3c>
D:\STM32\Program\1.11_Odchudzanie\um0427\FWLib\library\src/stm32f10x_tim.c:221
  38:	7a0b      	ldrb	r3, [r1, #8]
  3a:	8603      	strh	r3, [r0, #48]
D:\STM32\Program\1.11_Odchudzanie\um0427\FWLib\library\src/stm32f10x_tim.c:223
  3c:	b002      	add	sp, #8
  3e:	4770      	bx	lr
  40:	40012c00 	.word	0x40012c00
Disassembly of section .text.TIM_OC1Init:

00000000 <TIM_OC1Init>:
TIM_OC1Init():
D:\STM32\Program\1.11_Odchudzanie\um0427\FWLib\library\src/stm32f10x_tim.c:248
   0:	8c03      	ldrh	r3, [r0, #32]
D:\STM32\Program\1.11_Odchudzanie\um0427\FWLib\library\src/stm32f10x_tim.c:238
   2:	b573      	push	{r0, r1, r4, r5, r6, lr}
D:\STM32\Program\1.11_Odchudzanie\um0427\FWLib\library\src/stm32f10x_tim.c:248
   4:	f023 0301 	bic.w	r3, r3, #1	; 0x1
   8:	041b      	lsls	r3, r3, #16
   a:	0c1b      	lsrs	r3, r3, #16
   c:	8403      	strh	r3, [r0, #32]
D:\STM32\Program\1.11_Odchudzanie\um0427\FWLib\library\src/stm32f10x_tim.c:238
   e:	460c      	mov	r4, r1
D:\STM32\Program\1.11_Odchudzanie\um0427\FWLib\library\src/stm32f10x_tim.c:251
  10:	8c01      	ldrh	r1, [r0, #32]
D:\STM32\Program\1.11_Odchudzanie\um0427\FWLib\library\src/stm32f10x_tim.c:254
  12:	8883      	ldrh	r3, [r0, #4]
D:\STM32\Program\1.11_Odchudzanie\um0427\FWLib\library\src/stm32f10x_tim.c:269
  14:	8922      	ldrh	r2, [r4, #8]
D:\STM32\Program\1.11_Odchudzanie\um0427\FWLib\library\src/stm32f10x_tim.c:254
  16:	fa1f fc83 	uxth.w	ip, r3
D:\STM32\Program\1.11_Odchudzanie\um0427\FWLib\library\src/stm32f10x_tim.c:257
  1a:	8b03      	ldrh	r3, [r0, #24]
D:\STM32\Program\1.11_Odchudzanie\um0427\FWLib\library\src/stm32f10x_tim.c:266
  1c:	f021 0102 	bic.w	r1, r1, #2	; 0x2
D:\STM32\Program\1.11_Odchudzanie\um0427\FWLib\library\src/stm32f10x_tim.c:257
  20:	b29d      	uxth	r5, r3
D:\STM32\Program\1.11_Odchudzanie\um0427\FWLib\library\src/stm32f10x_tim.c:269
  22:	8863      	ldrh	r3, [r4, #2]
D:\STM32\Program\1.11_Odchudzanie\um0427\FWLib\library\src/stm32f10x_tim.c:266
  24:	0409      	lsls	r1, r1, #16
D:\STM32\Program\1.11_Odchudzanie\um0427\FWLib\library\src/stm32f10x_tim.c:269
  26:	4313      	orrs	r3, r2
D:\STM32\Program\1.11_Odchudzanie\um0427\FWLib\library\src/stm32f10x_tim.c:266
  28:	0c09      	lsrs	r1, r1, #16
D:\STM32\Program\1.11_Odchudzanie\um0427\FWLib\library\src/stm32f10x_tim.c:269
  2a:	b29b      	uxth	r3, r3
D:\STM32\Program\1.11_Odchudzanie\um0427\FWLib\library\src/stm32f10x_tim.c:272
  2c:	ea43 0e01 	orr.w	lr, r3, r1
D:\STM32\Program\1.11_Odchudzanie\um0427\FWLib\library\src/stm32f10x_tim.c:275
  30:	88e3      	ldrh	r3, [r4, #6]
D:\STM32\Program\1.11_Odchudzanie\um0427\FWLib\library\src/stm32f10x_tim.c:263
  32:	8826      	ldrh	r6, [r4, #0]
D:\STM32\Program\1.11_Odchudzanie\um0427\FWLib\library\src/stm32f10x_tim.c:275
  34:	8683      	strh	r3, [r0, #52]
D:\STM32\Program\1.11_Odchudzanie\um0427\FWLib\library\src/stm32f10x_tim.c:277
  36:	4b15      	ldr	r3, [pc, #84]	(8c <TIM_OC1Init+0x8c>)
D:\STM32\Program\1.11_Odchudzanie\um0427\FWLib\library\src/stm32f10x_tim.c:238
  38:	9001      	str	r0, [sp, #4]
D:\STM32\Program\1.11_Odchudzanie\um0427\FWLib\library\src/stm32f10x_tim.c:277
  3a:	4298      	cmp	r0, r3
  3c:	d003      	beq.n	46 <TIM_OC1Init+0x46>
  3e:	f503 6300 	add.w	r3, r3, #2048	; 0x800
  42:	4298      	cmp	r0, r3
  44:	d116      	bne.n	74 <TIM_OC1Init+0x74>
D:\STM32\Program\1.11_Odchudzanie\um0427\FWLib\library\src/stm32f10x_tim.c:288
  46:	8963      	ldrh	r3, [r4, #10]
D:\STM32\Program\1.11_Odchudzanie\um0427\FWLib\library\src/stm32f10x_tim.c:285
  48:	f64f 72f7 	movw	r2, #65527	; 0xfff7
  4c:	ea0e 0202 	and.w	r2, lr, r2
D:\STM32\Program\1.11_Odchudzanie\um0427\FWLib\library\src/stm32f10x_tim.c:288
  50:	431a      	orrs	r2, r3
D:\STM32\Program\1.11_Odchudzanie\um0427\FWLib\library\src/stm32f10x_tim.c:291
  52:	f64f 73fb 	movw	r3, #65531	; 0xfffb
  56:	ea02 0303 	and.w	r3, r2, r3
D:\STM32\Program\1.11_Odchudzanie\um0427\FWLib\library\src/stm32f10x_tim.c:294
  5a:	88a2      	ldrh	r2, [r4, #4]
D:\STM32\Program\1.11_Odchudzanie\um0427\FWLib\library\src/stm32f10x_tim.c:298
  5c:	f647 41ff 	movw	r1, #31999	; 0x7cff
D:\STM32\Program\1.11_Odchudzanie\um0427\FWLib\library\src/stm32f10x_tim.c:294
  60:	ea43 0e02 	orr.w	lr, r3, r2
D:\STM32\Program\1.11_Odchudzanie\um0427\FWLib\library\src/stm32f10x_tim.c:301
  64:	89e3      	ldrh	r3, [r4, #14]
  66:	89a2      	ldrh	r2, [r4, #12]
D:\STM32\Program\1.11_Odchudzanie\um0427\FWLib\library\src/stm32f10x_tim.c:298
  68:	ea0c 0101 	and.w	r1, ip, r1
D:\STM32\Program\1.11_Odchudzanie\um0427\FWLib\library\src/stm32f10x_tim.c:301
  6c:	4313      	orrs	r3, r2
  6e:	b29b      	uxth	r3, r3
D:\STM32\Program\1.11_Odchudzanie\um0427\FWLib\library\src/stm32f10x_tim.c:304
  70:	ea43 0c01 	orr.w	ip, r3, r1
D:\STM32\Program\1.11_Odchudzanie\um0427\FWLib\library\src/stm32f10x_tim.c:260
  74:	f64f 738f 	movw	r3, #65423	; 0xff8f
  78:	ea05 0303 	and.w	r3, r5, r3
D:\STM32\Program\1.11_Odchudzanie\um0427\FWLib\library\src/stm32f10x_tim.c:263
  7c:	4333      	orrs	r3, r6
D:\STM32\Program\1.11_Odchudzanie\um0427\FWLib\library\src/stm32f10x_tim.c:307
  7e:	f8a0 c004 	strh.w	ip, [r0, #4]
D:\STM32\Program\1.11_Odchudzanie\um0427\FWLib\library\src/stm32f10x_tim.c:310
  82:	8303      	strh	r3, [r0, #24]
D:\STM32\Program\1.11_Odchudzanie\um0427\FWLib\library\src/stm32f10x_tim.c:313
  84:	f8a0 e020 	strh.w	lr, [r0, #32]
D:\STM32\Program\1.11_Odchudzanie\um0427\FWLib\library\src/stm32f10x_tim.c:314
  88:	bd7c      	pop	{r2, r3, r4, r5, r6, pc}
  8a:	46c0      	nop			(mov r8, r8)
  8c:	40012c00 	.word	0x40012c00
Disassembly of section .text.TIM_OC2Init:

00000000 <TIM_OC2Init>:
TIM_OC2Init():
D:\STM32\Program\1.11_Odchudzanie\um0427\FWLib\library\src/stm32f10x_tim.c:339
   0:	8c03      	ldrh	r3, [r0, #32]
D:\STM32\Program\1.11_Odchudzanie\um0427\FWLib\library\src/stm32f10x_tim.c:329
   2:	b537      	push	{r0, r1, r2, r4, r5, lr}
D:\STM32\Program\1.11_Odchudzanie\um0427\FWLib\library\src/stm32f10x_tim.c:339
   4:	f023 0310 	bic.w	r3, r3, #16	; 0x10
   8:	041b      	lsls	r3, r3, #16
   a:	0c1b      	lsrs	r3, r3, #16
   c:	8403      	strh	r3, [r0, #32]
D:\STM32\Program\1.11_Odchudzanie\um0427\FWLib\library\src/stm32f10x_tim.c:342
   e:	8c03      	ldrh	r3, [r0, #32]
D:\STM32\Program\1.11_Odchudzanie\um0427\FWLib\library\src/stm32f10x_tim.c:345
  10:	8882      	ldrh	r2, [r0, #4]
D:\STM32\Program\1.11_Odchudzanie\um0427\FWLib\library\src/stm32f10x_tim.c:357
  12:	f023 0320 	bic.w	r3, r3, #32	; 0x20
D:\STM32\Program\1.11_Odchudzanie\um0427\FWLib\library\src/stm32f10x_tim.c:345
  16:	fa1f fc82 	uxth.w	ip, r2
D:\STM32\Program\1.11_Odchudzanie\um0427\FWLib\library\src/stm32f10x_tim.c:348
  1a:	8b02      	ldrh	r2, [r0, #24]
D:\STM32\Program\1.11_Odchudzanie\um0427\FWLib\library\src/stm32f10x_tim.c:357
  1c:	041b      	lsls	r3, r3, #16
D:\STM32\Program\1.11_Odchudzanie\um0427\FWLib\library\src/stm32f10x_tim.c:348
  1e:	b294      	uxth	r4, r2
D:\STM32\Program\1.11_Odchudzanie\um0427\FWLib\library\src/stm32f10x_tim.c:360
  20:	890a      	ldrh	r2, [r1, #8]
D:\STM32\Program\1.11_Odchudzanie\um0427\FWLib\library\src/stm32f10x_tim.c:357
  22:	0c1b      	lsrs	r3, r3, #16
D:\STM32\Program\1.11_Odchudzanie\um0427\FWLib\library\src/stm32f10x_tim.c:360
  24:	ea43 1302 	orr.w	r3, r3, r2, lsl #4
D:\STM32\Program\1.11_Odchudzanie\um0427\FWLib\library\src/stm32f10x_tim.c:363
  28:	884a      	ldrh	r2, [r1, #2]
D:\STM32\Program\1.11_Odchudzanie\um0427\FWLib\library\src/stm32f10x_tim.c:360
  2a:	b29b      	uxth	r3, r3
D:\STM32\Program\1.11_Odchudzanie\um0427\FWLib\library\src/stm32f10x_tim.c:363
  2c:	ea43 1302 	orr.w	r3, r3, r2, lsl #4
  30:	fa1f fe83 	uxth.w	lr, r3
D:\STM32\Program\1.11_Odchudzanie\um0427\FWLib\library\src/stm32f10x_tim.c:366
  34:	88cb      	ldrh	r3, [r1, #6]
D:\STM32\Program\1.11_Odchudzanie\um0427\FWLib\library\src/stm32f10x_tim.c:354
  36:	880d      	ldrh	r5, [r1, #0]
D:\STM32\Program\1.11_Odchudzanie\um0427\FWLib\library\src/stm32f10x_tim.c:366
  38:	8703      	strh	r3, [r0, #56]
D:\STM32\Program\1.11_Odchudzanie\um0427\FWLib\library\src/stm32f10x_tim.c:368
  3a:	4b19      	ldr	r3, [pc, #100]	(a0 <TIM_OC2Init+0xa0>)
D:\STM32\Program\1.11_Odchudzanie\um0427\FWLib\library\src/stm32f10x_tim.c:329
  3c:	9001      	str	r0, [sp, #4]
D:\STM32\Program\1.11_Odchudzanie\um0427\FWLib\library\src/stm32f10x_tim.c:368
  3e:	4298      	cmp	r0, r3
  40:	d003      	beq.n	4a <TIM_OC2Init+0x4a>
  42:	f503 6300 	add.w	r3, r3, #2048	; 0x800
  46:	4298      	cmp	r0, r3
  48:	d11c      	bne.n	84 <TIM_OC2Init+0x84>
D:\STM32\Program\1.11_Odchudzanie\um0427\FWLib\library\src/stm32f10x_tim.c:379
  4a:	894b      	ldrh	r3, [r1, #10]
D:\STM32\Program\1.11_Odchudzanie\um0427\FWLib\library\src/stm32f10x_tim.c:376
  4c:	f64f 727f 	movw	r2, #65407	; 0xff7f
  50:	ea0e 0202 	and.w	r2, lr, r2
D:\STM32\Program\1.11_Odchudzanie\um0427\FWLib\library\src/stm32f10x_tim.c:379
  54:	ea42 1203 	orr.w	r2, r2, r3, lsl #4
D:\STM32\Program\1.11_Odchudzanie\um0427\FWLib\library\src/stm32f10x_tim.c:382
  58:	f64f 73bf 	movw	r3, #65471	; 0xffbf
  5c:	ea02 0303 	and.w	r3, r2, r3
D:\STM32\Program\1.11_Odchudzanie\um0427\FWLib\library\src/stm32f10x_tim.c:385
  60:	888a      	ldrh	r2, [r1, #4]
  62:	ea43 1302 	orr.w	r3, r3, r2, lsl #4
  66:	fa1f fe83 	uxth.w	lr, r3
D:\STM32\Program\1.11_Odchudzanie\um0427\FWLib\library\src/stm32f10x_tim.c:392
  6a:	898a      	ldrh	r2, [r1, #12]
D:\STM32\Program\1.11_Odchudzanie\um0427\FWLib\library\src/stm32f10x_tim.c:389
  6c:	f247 33ff 	movw	r3, #29695	; 0x73ff
  70:	ea0c 0303 	and.w	r3, ip, r3
D:\STM32\Program\1.11_Odchudzanie\um0427\FWLib\library\src/stm32f10x_tim.c:392
  74:	ea43 0382 	orr.w	r3, r3, r2, lsl #2
D:\STM32\Program\1.11_Odchudzanie\um0427\FWLib\library\src/stm32f10x_tim.c:395
  78:	89ca      	ldrh	r2, [r1, #14]
D:\STM32\Program\1.11_Odchudzanie\um0427\FWLib\library\src/stm32f10x_tim.c:392
  7a:	b29b      	uxth	r3, r3
D:\STM32\Program\1.11_Odchudzanie\um0427\FWLib\library\src/stm32f10x_tim.c:395
  7c:	ea43 0382 	orr.w	r3, r3, r2, lsl #2
  80:	fa1f fc83 	uxth.w	ip, r3
D:\STM32\Program\1.11_Odchudzanie\um0427\FWLib\library\src/stm32f10x_tim.c:351
  84:	f648 73ff 	movw	r3, #36863	; 0x8fff
  88:	ea04 0303 	and.w	r3, r4, r3
D:\STM32\Program\1.11_Odchudzanie\um0427\FWLib\library\src/stm32f10x_tim.c:354
  8c:	ea43 2305 	orr.w	r3, r3, r5, lsl #8
  90:	b29b      	uxth	r3, r3
D:\STM32\Program\1.11_Odchudzanie\um0427\FWLib\library\src/stm32f10x_tim.c:399
  92:	f8a0 c004 	strh.w	ip, [r0, #4]
D:\STM32\Program\1.11_Odchudzanie\um0427\FWLib\library\src/stm32f10x_tim.c:402
  96:	8303      	strh	r3, [r0, #24]
D:\STM32\Program\1.11_Odchudzanie\um0427\FWLib\library\src/stm32f10x_tim.c:405
  98:	f8a0 e020 	strh.w	lr, [r0, #32]
D:\STM32\Program\1.11_Odchudzanie\um0427\FWLib\library\src/stm32f10x_tim.c:406
  9c:	bd3e      	pop	{r1, r2, r3, r4, r5, pc}
  9e:	46c0      	nop			(mov r8, r8)
  a0:	40012c00 	.word	0x40012c00
Disassembly of section .text.TIM_OC3Init:

00000000 <TIM_OC3Init>:
TIM_OC3Init():
D:\STM32\Program\1.11_Odchudzanie\um0427\FWLib\library\src/stm32f10x_tim.c:431
   0:	8c03      	ldrh	r3, [r0, #32]
D:\STM32\Program\1.11_Odchudzanie\um0427\FWLib\library\src/stm32f10x_tim.c:421
   2:	b537      	push	{r0, r1, r2, r4, r5, lr}
D:\STM32\Program\1.11_Odchudzanie\um0427\FWLib\library\src/stm32f10x_tim.c:431
   4:	f423 7380 	bic.w	r3, r3, #256	; 0x100
   8:	041b      	lsls	r3, r3, #16
   a:	0c1b      	lsrs	r3, r3, #16
   c:	8403      	strh	r3, [r0, #32]
D:\STM32\Program\1.11_Odchudzanie\um0427\FWLib\library\src/stm32f10x_tim.c:434
   e:	8c03      	ldrh	r3, [r0, #32]
D:\STM32\Program\1.11_Odchudzanie\um0427\FWLib\library\src/stm32f10x_tim.c:437
  10:	8882      	ldrh	r2, [r0, #4]
D:\STM32\Program\1.11_Odchudzanie\um0427\FWLib\library\src/stm32f10x_tim.c:449
  12:	f423 7300 	bic.w	r3, r3, #512	; 0x200
D:\STM32\Program\1.11_Odchudzanie\um0427\FWLib\library\src/stm32f10x_tim.c:437
  16:	fa1f fc82 	uxth.w	ip, r2
D:\STM32\Program\1.11_Odchudzanie\um0427\FWLib\library\src/stm32f10x_tim.c:440
  1a:	8b82      	ldrh	r2, [r0, #28]
D:\STM32\Program\1.11_Odchudzanie\um0427\FWLib\library\src/stm32f10x_tim.c:449
  1c:	041b      	lsls	r3, r3, #16
D:\STM32\Program\1.11_Odchudzanie\um0427\FWLib\library\src/stm32f10x_tim.c:440
  1e:	b294      	uxth	r4, r2
D:\STM32\Program\1.11_Odchudzanie\um0427\FWLib\library\src/stm32f10x_tim.c:452
  20:	890a      	ldrh	r2, [r1, #8]
D:\STM32\Program\1.11_Odchudzanie\um0427\FWLib\library\src/stm32f10x_tim.c:449
  22:	0c1b      	lsrs	r3, r3, #16
D:\STM32\Program\1.11_Odchudzanie\um0427\FWLib\library\src/stm32f10x_tim.c:452
  24:	ea43 2302 	orr.w	r3, r3, r2, lsl #8
D:\STM32\Program\1.11_Odchudzanie\um0427\FWLib\library\src/stm32f10x_tim.c:455
  28:	884a      	ldrh	r2, [r1, #2]
D:\STM32\Program\1.11_Odchudzanie\um0427\FWLib\library\src/stm32f10x_tim.c:452
  2a:	b29b      	uxth	r3, r3
D:\STM32\Program\1.11_Odchudzanie\um0427\FWLib\library\src/stm32f10x_tim.c:455
  2c:	ea43 2302 	orr.w	r3, r3, r2, lsl #8
  30:	fa1f fe83 	uxth.w	lr, r3
D:\STM32\Program\1.11_Odchudzanie\um0427\FWLib\library\src/stm32f10x_tim.c:458
  34:	88cb      	ldrh	r3, [r1, #6]
D:\STM32\Program\1.11_Odchudzanie\um0427\FWLib\library\src/stm32f10x_tim.c:446
  36:	880d      	ldrh	r5, [r1, #0]
D:\STM32\Program\1.11_Odchudzanie\um0427\FWLib\library\src/stm32f10x_tim.c:458
  38:	8783      	strh	r3, [r0, #60]
D:\STM32\Program\1.11_Odchudzanie\um0427\FWLib\library\src/stm32f10x_tim.c:460
  3a:	4b18      	ldr	r3, [pc, #96]	(9c <TIM_OC3Init+0x9c>)
D:\STM32\Program\1.11_Odchudzanie\um0427\FWLib\library\src/stm32f10x_tim.c:421
  3c:	9001      	str	r0, [sp, #4]
D:\STM32\Program\1.11_Odchudzanie\um0427\FWLib\library\src/stm32f10x_tim.c:460
  3e:	4298      	cmp	r0, r3
  40:	d003      	beq.n	4a <TIM_OC3Init+0x4a>
  42:	f503 6300 	add.w	r3, r3, #2048	; 0x800
  46:	4298      	cmp	r0, r3
  48:	d11c      	bne.n	84 <TIM_OC3Init+0x84>
D:\STM32\Program\1.11_Odchudzanie\um0427\FWLib\library\src/stm32f10x_tim.c:471
  4a:	894b      	ldrh	r3, [r1, #10]
D:\STM32\Program\1.11_Odchudzanie\um0427\FWLib\library\src/stm32f10x_tim.c:468
  4c:	f24f 72ff 	movw	r2, #63487	; 0xf7ff
  50:	ea0e 0202 	and.w	r2, lr, r2
D:\STM32\Program\1.11_Odchudzanie\um0427\FWLib\library\src/stm32f10x_tim.c:471
  54:	ea42 2203 	orr.w	r2, r2, r3, lsl #8
D:\STM32\Program\1.11_Odchudzanie\um0427\FWLib\library\src/stm32f10x_tim.c:474
  58:	f64f 33ff 	movw	r3, #64511	; 0xfbff
  5c:	ea02 0303 	and.w	r3, r2, r3
D:\STM32\Program\1.11_Odchudzanie\um0427\FWLib\library\src/stm32f10x_tim.c:477
  60:	888a      	ldrh	r2, [r1, #4]
  62:	ea43 2302 	orr.w	r3, r3, r2, lsl #8
  66:	fa1f fe83 	uxth.w	lr, r3
D:\STM32\Program\1.11_Odchudzanie\um0427\FWLib\library\src/stm32f10x_tim.c:484
  6a:	898a      	ldrh	r2, [r1, #12]
D:\STM32\Program\1.11_Odchudzanie\um0427\FWLib\library\src/stm32f10x_tim.c:481
  6c:	f644 73ff 	movw	r3, #20479	; 0x4fff
  70:	ea0c 0303 	and.w	r3, ip, r3
D:\STM32\Program\1.11_Odchudzanie\um0427\FWLib\library\src/stm32f10x_tim.c:484
  74:	ea43 1302 	orr.w	r3, r3, r2, lsl #4
D:\STM32\Program\1.11_Odchudzanie\um0427\FWLib\library\src/stm32f10x_tim.c:487
  78:	89ca      	ldrh	r2, [r1, #14]
D:\STM32\Program\1.11_Odchudzanie\um0427\FWLib\library\src/stm32f10x_tim.c:484
  7a:	b29b      	uxth	r3, r3
D:\STM32\Program\1.11_Odchudzanie\um0427\FWLib\library\src/stm32f10x_tim.c:487
  7c:	ea43 1302 	orr.w	r3, r3, r2, lsl #4
  80:	fa1f fc83 	uxth.w	ip, r3
D:\STM32\Program\1.11_Odchudzanie\um0427\FWLib\library\src/stm32f10x_tim.c:443
  84:	f64f 738f 	movw	r3, #65423	; 0xff8f
  88:	ea04 0303 	and.w	r3, r4, r3
D:\STM32\Program\1.11_Odchudzanie\um0427\FWLib\library\src/stm32f10x_tim.c:446
  8c:	432b      	orrs	r3, r5
D:\STM32\Program\1.11_Odchudzanie\um0427\FWLib\library\src/stm32f10x_tim.c:491
  8e:	f8a0 c004 	strh.w	ip, [r0, #4]
D:\STM32\Program\1.11_Odchudzanie\um0427\FWLib\library\src/stm32f10x_tim.c:494
  92:	8383      	strh	r3, [r0, #28]
D:\STM32\Program\1.11_Odchudzanie\um0427\FWLib\library\src/stm32f10x_tim.c:497
  94:	f8a0 e020 	strh.w	lr, [r0, #32]
D:\STM32\Program\1.11_Odchudzanie\um0427\FWLib\library\src/stm32f10x_tim.c:498
  98:	bd3e      	pop	{r1, r2, r3, r4, r5, pc}
  9a:	46c0      	nop			(mov r8, r8)
  9c:	40012c00 	.word	0x40012c00
Disassembly of section .text.TIM_OC4Init:

00000000 <TIM_OC4Init>:
TIM_OC4Init():
D:\STM32\Program\1.11_Odchudzanie\um0427\FWLib\library\src/stm32f10x_tim.c:523
   0:	8c03      	ldrh	r3, [r0, #32]
D:\STM32\Program\1.11_Odchudzanie\um0427\FWLib\library\src/stm32f10x_tim.c:513
   2:	b573      	push	{r0, r1, r4, r5, r6, lr}
D:\STM32\Program\1.11_Odchudzanie\um0427\FWLib\library\src/stm32f10x_tim.c:523
   4:	f423 5380 	bic.w	r3, r3, #4096	; 0x1000
   8:	041b      	lsls	r3, r3, #16
   a:	0c1b      	lsrs	r3, r3, #16
   c:	8403      	strh	r3, [r0, #32]
D:\STM32\Program\1.11_Odchudzanie\um0427\FWLib\library\src/stm32f10x_tim.c:526
   e:	8c03      	ldrh	r3, [r0, #32]
D:\STM32\Program\1.11_Odchudzanie\um0427\FWLib\library\src/stm32f10x_tim.c:513
  10:	460a      	mov	r2, r1
D:\STM32\Program\1.11_Odchudzanie\um0427\FWLib\library\src/stm32f10x_tim.c:526
  12:	b29e      	uxth	r6, r3
D:\STM32\Program\1.11_Odchudzanie\um0427\FWLib\library\src/stm32f10x_tim.c:529
  14:	8883      	ldrh	r3, [r0, #4]
D:\STM32\Program\1.11_Odchudzanie\um0427\FWLib\library\src/stm32f10x_tim.c:538
  16:	f8b2 c000 	ldrh.w	ip, [r2]
D:\STM32\Program\1.11_Odchudzanie\um0427\FWLib\library\src/stm32f10x_tim.c:529
  1a:	b299      	uxth	r1, r3
D:\STM32\Program\1.11_Odchudzanie\um0427\FWLib\library\src/stm32f10x_tim.c:532
  1c:	8b83      	ldrh	r3, [r0, #28]
D:\STM32\Program\1.11_Odchudzanie\um0427\FWLib\library\src/stm32f10x_tim.c:544
  1e:	8914      	ldrh	r4, [r2, #8]
D:\STM32\Program\1.11_Odchudzanie\um0427\FWLib\library\src/stm32f10x_tim.c:532
  20:	fa1f fe83 	uxth.w	lr, r3
D:\STM32\Program\1.11_Odchudzanie\um0427\FWLib\library\src/stm32f10x_tim.c:550
  24:	88d3      	ldrh	r3, [r2, #6]
D:\STM32\Program\1.11_Odchudzanie\um0427\FWLib\library\src/stm32f10x_tim.c:547
  26:	8855      	ldrh	r5, [r2, #2]
D:\STM32\Program\1.11_Odchudzanie\um0427\FWLib\library\src/stm32f10x_tim.c:550
  28:	f8a0 3040 	strh.w	r3, [r0, #64]
D:\STM32\Program\1.11_Odchudzanie\um0427\FWLib\library\src/stm32f10x_tim.c:552
  2c:	4b11      	ldr	r3, [pc, #68]	(74 <TIM_OC4Init+0x74>)
D:\STM32\Program\1.11_Odchudzanie\um0427\FWLib\library\src/stm32f10x_tim.c:513
  2e:	9001      	str	r0, [sp, #4]
D:\STM32\Program\1.11_Odchudzanie\um0427\FWLib\library\src/stm32f10x_tim.c:552
  30:	4298      	cmp	r0, r3
  32:	d003      	beq.n	3c <TIM_OC4Init+0x3c>
  34:	f503 6300 	add.w	r3, r3, #2048	; 0x800
  38:	4298      	cmp	r0, r3
  3a:	d105      	bne.n	48 <TIM_OC4Init+0x48>
D:\STM32\Program\1.11_Odchudzanie\um0427\FWLib\library\src/stm32f10x_tim.c:557
  3c:	048b      	lsls	r3, r1, #18
D:\STM32\Program\1.11_Odchudzanie\um0427\FWLib\library\src/stm32f10x_tim.c:560
  3e:	8992      	ldrh	r2, [r2, #12]
D:\STM32\Program\1.11_Odchudzanie\um0427\FWLib\library\src/stm32f10x_tim.c:557
  40:	0c9b      	lsrs	r3, r3, #18
D:\STM32\Program\1.11_Odchudzanie\um0427\FWLib\library\src/stm32f10x_tim.c:560
  42:	ea43 1382 	orr.w	r3, r3, r2, lsl #6
  46:	b299      	uxth	r1, r3
D:\STM32\Program\1.11_Odchudzanie\um0427\FWLib\library\src/stm32f10x_tim.c:535
  48:	f648 73ff 	movw	r3, #36863	; 0x8fff
  4c:	ea0e 0303 	and.w	r3, lr, r3
D:\STM32\Program\1.11_Odchudzanie\um0427\FWLib\library\src/stm32f10x_tim.c:538
  50:	ea43 230c 	orr.w	r3, r3, ip, lsl #8
  54:	b29b      	uxth	r3, r3
D:\STM32\Program\1.11_Odchudzanie\um0427\FWLib\library\src/stm32f10x_tim.c:564
  56:	8081      	strh	r1, [r0, #4]
D:\STM32\Program\1.11_Odchudzanie\um0427\FWLib\library\src/stm32f10x_tim.c:567
  58:	8383      	strh	r3, [r0, #28]
D:\STM32\Program\1.11_Odchudzanie\um0427\FWLib\library\src/stm32f10x_tim.c:541
  5a:	f64d 73ff 	movw	r3, #57343	; 0xdfff
  5e:	ea06 0303 	and.w	r3, r6, r3
D:\STM32\Program\1.11_Odchudzanie\um0427\FWLib\library\src/stm32f10x_tim.c:544
  62:	ea43 3304 	orr.w	r3, r3, r4, lsl #12
  66:	b29b      	uxth	r3, r3
D:\STM32\Program\1.11_Odchudzanie\um0427\FWLib\library\src/stm32f10x_tim.c:547
  68:	ea43 3305 	orr.w	r3, r3, r5, lsl #12
  6c:	b29b      	uxth	r3, r3
D:\STM32\Program\1.11_Odchudzanie\um0427\FWLib\library\src/stm32f10x_tim.c:570
  6e:	8403      	strh	r3, [r0, #32]
D:\STM32\Program\1.11_Odchudzanie\um0427\FWLib\library\src/stm32f10x_tim.c:571
  70:	bd7c      	pop	{r2, r3, r4, r5, r6, pc}
  72:	46c0      	nop			(mov r8, r8)
  74:	40012c00 	.word	0x40012c00
Disassembly of section .text.TIM_BDTRConfig:

00000000 <TIM_BDTRConfig>:
TIM_BDTRConfig():
D:\STM32\Program\1.11_Odchudzanie\um0427\FWLib\library\src/stm32f10x_tim.c:735
   0:	880a      	ldrh	r2, [r1, #0]
   2:	884b      	ldrh	r3, [r1, #2]
   4:	4313      	orrs	r3, r2
   6:	888a      	ldrh	r2, [r1, #4]
   8:	4313      	orrs	r3, r2
   a:	88ca      	ldrh	r2, [r1, #6]
   c:	4313      	orrs	r3, r2
   e:	890a      	ldrh	r2, [r1, #8]
  10:	4313      	orrs	r3, r2
  12:	894a      	ldrh	r2, [r1, #10]
  14:	4313      	orrs	r3, r2
  16:	898a      	ldrh	r2, [r1, #12]
  18:	4313      	orrs	r3, r2
  1a:	b29b      	uxth	r3, r3
  1c:	f8a0 3044 	strh.w	r3, [r0, #68]
D:\STM32\Program\1.11_Odchudzanie\um0427\FWLib\library\src/stm32f10x_tim.c:740
  20:	4770      	bx	lr
  22:	46c0      	nop			(mov r8, r8)
Disassembly of section .text.TIM_TimeBaseStructInit:

00000000 <TIM_TimeBaseStructInit>:
TIM_TimeBaseStructInit():
D:\STM32\Program\1.11_Odchudzanie\um0427\FWLib\library\src/stm32f10x_tim.c:753
   0:	f04f 33ff 	mov.w	r3, #4294967295	; 0xffffffff
   4:	8083      	strh	r3, [r0, #4]
D:\STM32\Program\1.11_Odchudzanie\um0427\FWLib\library\src/stm32f10x_tim.c:754
   6:	2300      	movs	r3, #0
   8:	8003      	strh	r3, [r0, #0]
D:\STM32\Program\1.11_Odchudzanie\um0427\FWLib\library\src/stm32f10x_tim.c:755
   a:	80c3      	strh	r3, [r0, #6]
D:\STM32\Program\1.11_Odchudzanie\um0427\FWLib\library\src/stm32f10x_tim.c:756
   c:	8043      	strh	r3, [r0, #2]
D:\STM32\Program\1.11_Odchudzanie\um0427\FWLib\library\src/stm32f10x_tim.c:757
   e:	7203      	strb	r3, [r0, #8]
D:\STM32\Program\1.11_Odchudzanie\um0427\FWLib\library\src/stm32f10x_tim.c:758
  10:	4770      	bx	lr
  12:	46c0      	nop			(mov r8, r8)
Disassembly of section .text.TIM_OCStructInit:

00000000 <TIM_OCStructInit>:
TIM_OCStructInit():
D:\STM32\Program\1.11_Odchudzanie\um0427\FWLib\library\src/stm32f10x_tim.c:771
   0:	2300      	movs	r3, #0
   2:	8003      	strh	r3, [r0, #0]
D:\STM32\Program\1.11_Odchudzanie\um0427\FWLib\library\src/stm32f10x_tim.c:772
   4:	8043      	strh	r3, [r0, #2]
D:\STM32\Program\1.11_Odchudzanie\um0427\FWLib\library\src/stm32f10x_tim.c:773
   6:	8083      	strh	r3, [r0, #4]
D:\STM32\Program\1.11_Odchudzanie\um0427\FWLib\library\src/stm32f10x_tim.c:774
   8:	80c3      	strh	r3, [r0, #6]
D:\STM32\Program\1.11_Odchudzanie\um0427\FWLib\library\src/stm32f10x_tim.c:775
   a:	8103      	strh	r3, [r0, #8]
D:\STM32\Program\1.11_Odchudzanie\um0427\FWLib\library\src/stm32f10x_tim.c:776
   c:	8143      	strh	r3, [r0, #10]
D:\STM32\Program\1.11_Odchudzanie\um0427\FWLib\library\src/stm32f10x_tim.c:777
   e:	8183      	strh	r3, [r0, #12]
D:\STM32\Program\1.11_Odchudzanie\um0427\FWLib\library\src/stm32f10x_tim.c:778
  10:	81c3      	strh	r3, [r0, #14]
D:\STM32\Program\1.11_Odchudzanie\um0427\FWLib\library\src/stm32f10x_tim.c:779
  12:	4770      	bx	lr
Disassembly of section .text.TIM_ICStructInit:

00000000 <TIM_ICStructInit>:
TIM_ICStructInit():
D:\STM32\Program\1.11_Odchudzanie\um0427\FWLib\library\src/stm32f10x_tim.c:792
   0:	2300      	movs	r3, #0
D:\STM32\Program\1.11_Odchudzanie\um0427\FWLib\library\src/stm32f10x_tim.c:794
   2:	f04f 0201 	mov.w	r2, #1	; 0x1
D:\STM32\Program\1.11_Odchudzanie\um0427\FWLib\library\src/stm32f10x_tim.c:792
   6:	8003      	strh	r3, [r0, #0]
D:\STM32\Program\1.11_Odchudzanie\um0427\FWLib\library\src/stm32f10x_tim.c:793
   8:	8043      	strh	r3, [r0, #2]
D:\STM32\Program\1.11_Odchudzanie\um0427\FWLib\library\src/stm32f10x_tim.c:794
   a:	8082      	strh	r2, [r0, #4]
D:\STM32\Program\1.11_Odchudzanie\um0427\FWLib\library\src/stm32f10x_tim.c:795
   c:	80c3      	strh	r3, [r0, #6]
D:\STM32\Program\1.11_Odchudzanie\um0427\FWLib\library\src/stm32f10x_tim.c:796
   e:	8103      	strh	r3, [r0, #8]
D:\STM32\Program\1.11_Odchudzanie\um0427\FWLib\library\src/stm32f10x_tim.c:797
  10:	4770      	bx	lr
  12:	46c0      	nop			(mov r8, r8)
Disassembly of section .text.TIM_BDTRStructInit:

00000000 <TIM_BDTRStructInit>:
TIM_BDTRStructInit():
D:\STM32\Program\1.11_Odchudzanie\um0427\FWLib\library\src/stm32f10x_tim.c:810
   0:	2300      	movs	r3, #0
   2:	8003      	strh	r3, [r0, #0]
D:\STM32\Program\1.11_Odchudzanie\um0427\FWLib\library\src/stm32f10x_tim.c:811
   4:	8043      	strh	r3, [r0, #2]
D:\STM32\Program\1.11_Odchudzanie\um0427\FWLib\library\src/stm32f10x_tim.c:812
   6:	8083      	strh	r3, [r0, #4]
D:\STM32\Program\1.11_Odchudzanie\um0427\FWLib\library\src/stm32f10x_tim.c:813
   8:	80c3      	strh	r3, [r0, #6]
D:\STM32\Program\1.11_Odchudzanie\um0427\FWLib\library\src/stm32f10x_tim.c:814
   a:	8103      	strh	r3, [r0, #8]
D:\STM32\Program\1.11_Odchudzanie\um0427\FWLib\library\src/stm32f10x_tim.c:815
   c:	8143      	strh	r3, [r0, #10]
D:\STM32\Program\1.11_Odchudzanie\um0427\FWLib\library\src/stm32f10x_tim.c:816
   e:	8183      	strh	r3, [r0, #12]
D:\STM32\Program\1.11_Odchudzanie\um0427\FWLib\library\src/stm32f10x_tim.c:817
  10:	4770      	bx	lr
  12:	46c0      	nop			(mov r8, r8)
Disassembly of section .text.TIM_Cmd:

00000000 <TIM_Cmd>:
TIM_Cmd():
D:\STM32\Program\1.11_Odchudzanie\um0427\FWLib\library\src/stm32f10x_tim.c:834
   0:	b121      	cbz	r1, c <TIM_Cmd+0xc>
D:\STM32\Program\1.11_Odchudzanie\um0427\FWLib\library\src/stm32f10x_tim.c:837
   2:	8803      	ldrh	r3, [r0, #0]
   4:	b29b      	uxth	r3, r3
   6:	f043 0301 	orr.w	r3, r3, #1	; 0x1
   a:	e004      	b.n	16 <TIM_Cmd+0x16>
D:\STM32\Program\1.11_Odchudzanie\um0427\FWLib\library\src/stm32f10x_tim.c:842
   c:	8803      	ldrh	r3, [r0, #0]
   e:	f023 0301 	bic.w	r3, r3, #1	; 0x1
  12:	059b      	lsls	r3, r3, #22
  14:	0d9b      	lsrs	r3, r3, #22
  16:	8003      	strh	r3, [r0, #0]
D:\STM32\Program\1.11_Odchudzanie\um0427\FWLib\library\src/stm32f10x_tim.c:844
  18:	4770      	bx	lr
  1a:	46c0      	nop			(mov r8, r8)
Disassembly of section .text.TIM_CtrlPWMOutputs:

00000000 <TIM_CtrlPWMOutputs>:
TIM_CtrlPWMOutputs():
D:\STM32\Program\1.11_Odchudzanie\um0427\FWLib\library\src/stm32f10x_tim.c:861
   0:	b139      	cbz	r1, 12 <TIM_CtrlPWMOutputs+0x12>
D:\STM32\Program\1.11_Odchudzanie\um0427\FWLib\library\src/stm32f10x_tim.c:864
   2:	f8b0 3044 	ldrh.w	r3, [r0, #68]
   6:	ea6f 4343 	mvn.w	r3, r3, lsl #17
   a:	ea6f 4353 	mvn.w	r3, r3, lsr #17
   e:	b29b      	uxth	r3, r3
  10:	e003      	b.n	1a <TIM_CtrlPWMOutputs+0x1a>
D:\STM32\Program\1.11_Odchudzanie\um0427\FWLib\library\src/stm32f10x_tim.c:869
  12:	f8b0 3044 	ldrh.w	r3, [r0, #68]
  16:	045b      	lsls	r3, r3, #17
  18:	0c5b      	lsrs	r3, r3, #17
  1a:	f8a0 3044 	strh.w	r3, [r0, #68]
D:\STM32\Program\1.11_Odchudzanie\um0427\FWLib\library\src/stm32f10x_tim.c:871
  1e:	4770      	bx	lr
Disassembly of section .text.TIM_ITConfig:

00000000 <TIM_ITConfig>:
TIM_ITConfig():
D:\STM32\Program\1.11_Odchudzanie\um0427\FWLib\library\src/stm32f10x_tim.c:901
   0:	b122      	cbz	r2, c <TIM_ITConfig+0xc>
D:\STM32\Program\1.11_Odchudzanie\um0427\FWLib\library\src/stm32f10x_tim.c:904
   2:	8983      	ldrh	r3, [r0, #12]
   4:	b29b      	uxth	r3, r3
   6:	ea41 0303 	orr.w	r3, r1, r3
   a:	e003      	b.n	14 <TIM_ITConfig+0x14>
D:\STM32\Program\1.11_Odchudzanie\um0427\FWLib\library\src/stm32f10x_tim.c:909
   c:	8983      	ldrh	r3, [r0, #12]
   e:	b29b      	uxth	r3, r3
  10:	ea23 0301 	bic.w	r3, r3, r1
  14:	8183      	strh	r3, [r0, #12]
D:\STM32\Program\1.11_Odchudzanie\um0427\FWLib\library\src/stm32f10x_tim.c:911
  16:	4770      	bx	lr
Disassembly of section .text.TIM_GenerateEvent:

00000000 <TIM_GenerateEvent>:
TIM_GenerateEvent():
D:\STM32\Program\1.11_Odchudzanie\um0427\FWLib\library\src/stm32f10x_tim.c:936
   0:	8281      	strh	r1, [r0, #20]
D:\STM32\Program\1.11_Odchudzanie\um0427\FWLib\library\src/stm32f10x_tim.c:937
   2:	4770      	bx	lr
Disassembly of section .text.TIM_DMAConfig:

00000000 <TIM_DMAConfig>:
TIM_DMAConfig():
D:\STM32\Program\1.11_Odchudzanie\um0427\FWLib\library\src/stm32f10x_tim.c:967
   0:	430a      	orrs	r2, r1
   2:	f8a0 2048 	strh.w	r2, [r0, #72]
D:\STM32\Program\1.11_Odchudzanie\um0427\FWLib\library\src/stm32f10x_tim.c:968
   6:	4770      	bx	lr
Disassembly of section .text.TIM_DMACmd:

00000000 <TIM_DMACmd>:
TIM_DMACmd():
D:\STM32\Program\1.11_Odchudzanie\um0427\FWLib\library\src/stm32f10x_tim.c:996
   0:	b122      	cbz	r2, c <TIM_DMACmd+0xc>
D:\STM32\Program\1.11_Odchudzanie\um0427\FWLib\library\src/stm32f10x_tim.c:999
   2:	8983      	ldrh	r3, [r0, #12]
   4:	b29b      	uxth	r3, r3
   6:	ea41 0303 	orr.w	r3, r1, r3
   a:	e003      	b.n	14 <TIM_DMACmd+0x14>
D:\STM32\Program\1.11_Odchudzanie\um0427\FWLib\library\src/stm32f10x_tim.c:1004
   c:	8983      	ldrh	r3, [r0, #12]
   e:	b29b      	uxth	r3, r3
  10:	ea23 0301 	bic.w	r3, r3, r1
  14:	8183      	strh	r3, [r0, #12]
D:\STM32\Program\1.11_Odchudzanie\um0427\FWLib\library\src/stm32f10x_tim.c:1006
  16:	4770      	bx	lr
Disassembly of section .text.TIM_InternalClockConfig:

00000000 <TIM_InternalClockConfig>:
TIM_InternalClockConfig():
D:\STM32\Program\1.11_Odchudzanie\um0427\FWLib\library\src/stm32f10x_tim.c:1022
   0:	8903      	ldrh	r3, [r0, #8]
   2:	f023 0307 	bic.w	r3, r3, #7	; 0x7
   6:	041b      	lsls	r3, r3, #16
   8:	0c1b      	lsrs	r3, r3, #16
   a:	8103      	strh	r3, [r0, #8]
D:\STM32\Program\1.11_Odchudzanie\um0427\FWLib\library\src/stm32f10x_tim.c:1023
   c:	4770      	bx	lr
   e:	46c0      	nop			(mov r8, r8)
Disassembly of section .text.TIM_ETRConfig:

00000000 <TIM_ETRConfig>:
TIM_ETRConfig():
D:\STM32\Program\1.11_Odchudzanie\um0427\FWLib\library\src/stm32f10x_tim.c:1203
   0:	b510      	push	{r4, lr}
D:\STM32\Program\1.11_Odchudzanie\um0427\FWLib\library\src/stm32f10x_tim.c:1212
   2:	8904      	ldrh	r4, [r0, #8]
D:\STM32\Program\1.11_Odchudzanie\um0427\FWLib\library\src/stm32f10x_tim.c:1218
   4:	b2e4      	uxtb	r4, r4
   6:	4321      	orrs	r1, r4
   8:	430a      	orrs	r2, r1
   a:	ea42 2203 	orr.w	r2, r2, r3, lsl #8
   e:	b292      	uxth	r2, r2
D:\STM32\Program\1.11_Odchudzanie\um0427\FWLib\library\src/stm32f10x_tim.c:1221
  10:	8102      	strh	r2, [r0, #8]
D:\STM32\Program\1.11_Odchudzanie\um0427\FWLib\library\src/stm32f10x_tim.c:1222
  12:	bd10      	pop	{r4, pc}
Disassembly of section .text.TIM_ETRClockMode2Config:

00000000 <TIM_ETRClockMode2Config>:
TIM_ETRClockMode2Config():
D:\STM32\Program\1.11_Odchudzanie\um0427\FWLib\library\src/stm32f10x_tim.c:1167
   0:	b510      	push	{r4, lr}
   2:	4604      	mov	r4, r0
D:\STM32\Program\1.11_Odchudzanie\um0427\FWLib\library\src/stm32f10x_tim.c:1175
   4:	f7ff fffe 	bl	0 <TIM_ETRClockMode2Config>
D:\STM32\Program\1.11_Odchudzanie\um0427\FWLib\library\src/stm32f10x_tim.c:1178
   8:	8923      	ldrh	r3, [r4, #8]
   a:	b29b      	uxth	r3, r3
   c:	f443 4380 	orr.w	r3, r3, #16384	; 0x4000
  10:	8123      	strh	r3, [r4, #8]
D:\STM32\Program\1.11_Odchudzanie\um0427\FWLib\library\src/stm32f10x_tim.c:1179
  12:	bd10      	pop	{r4, pc}
Disassembly of section .text.TIM_ETRClockMode1Config:

00000000 <TIM_ETRClockMode1Config>:
TIM_ETRClockMode1Config():
D:\STM32\Program\1.11_Odchudzanie\um0427\FWLib\library\src/stm32f10x_tim.c:1117
   0:	b510      	push	{r4, lr}
   2:	4604      	mov	r4, r0
D:\STM32\Program\1.11_Odchudzanie\um0427\FWLib\library\src/stm32f10x_tim.c:1127
   4:	f7ff fffe 	bl	0 <TIM_ETRClockMode1Config>
D:\STM32\Program\1.11_Odchudzanie\um0427\FWLib\library\src/stm32f10x_tim.c:1130
   8:	8923      	ldrh	r3, [r4, #8]
D:\STM32\Program\1.11_Odchudzanie\um0427\FWLib\library\src/stm32f10x_tim.c:1135
   a:	f023 0377 	bic.w	r3, r3, #119	; 0x77
   e:	041b      	lsls	r3, r3, #16
  10:	0c1b      	lsrs	r3, r3, #16
D:\STM32\Program\1.11_Odchudzanie\um0427\FWLib\library\src/stm32f10x_tim.c:1139
  12:	f043 0377 	orr.w	r3, r3, #119	; 0x77
D:\STM32\Program\1.11_Odchudzanie\um0427\FWLib\library\src/stm32f10x_tim.c:1142
  16:	8123      	strh	r3, [r4, #8]
D:\STM32\Program\1.11_Odchudzanie\um0427\FWLib\library\src/stm32f10x_tim.c:1143
  18:	bd10      	pop	{r4, pc}
  1a:	46c0      	nop			(mov r8, r8)
Disassembly of section .text.TIM_PrescalerConfig:

00000000 <TIM_PrescalerConfig>:
TIM_PrescalerConfig():
D:\STM32\Program\1.11_Odchudzanie\um0427\FWLib\library\src/stm32f10x_tim.c:1245
   0:	8501      	strh	r1, [r0, #40]
D:\STM32\Program\1.11_Odchudzanie\um0427\FWLib\library\src/stm32f10x_tim.c:1248
   2:	8282      	strh	r2, [r0, #20]
D:\STM32\Program\1.11_Odchudzanie\um0427\FWLib\library\src/stm32f10x_tim.c:1249
   4:	4770      	bx	lr
   6:	46c0      	nop			(mov r8, r8)
Disassembly of section .text.TIM_CounterModeConfig:

00000000 <TIM_CounterModeConfig>:
TIM_CounterModeConfig():
D:\STM32\Program\1.11_Odchudzanie\um0427\FWLib\library\src/stm32f10x_tim.c:1274
   0:	8803      	ldrh	r3, [r0, #0]
D:\STM32\Program\1.11_Odchudzanie\um0427\FWLib\library\src/stm32f10x_tim.c:1277
   2:	f023 0370 	bic.w	r3, r3, #112	; 0x70
   6:	059b      	lsls	r3, r3, #22
   8:	0d9b      	lsrs	r3, r3, #22
D:\STM32\Program\1.11_Odchudzanie\um0427\FWLib\library\src/stm32f10x_tim.c:1280
   a:	4319      	orrs	r1, r3
D:\STM32\Program\1.11_Odchudzanie\um0427\FWLib\library\src/stm32f10x_tim.c:1283
   c:	8001      	strh	r1, [r0, #0]
D:\STM32\Program\1.11_Odchudzanie\um0427\FWLib\library\src/stm32f10x_tim.c:1284
   e:	4770      	bx	lr
Disassembly of section .text.TIM_SelectInputTrigger:

00000000 <TIM_SelectInputTrigger>:
TIM_SelectInputTrigger():
D:\STM32\Program\1.11_Odchudzanie\um0427\FWLib\library\src/stm32f10x_tim.c:1313
   0:	8903      	ldrh	r3, [r0, #8]
D:\STM32\Program\1.11_Odchudzanie\um0427\FWLib\library\src/stm32f10x_tim.c:1316
   2:	f023 0370 	bic.w	r3, r3, #112	; 0x70
   6:	041b      	lsls	r3, r3, #16
   8:	0c1b      	lsrs	r3, r3, #16
D:\STM32\Program\1.11_Odchudzanie\um0427\FWLib\library\src/stm32f10x_tim.c:1319
   a:	4319      	orrs	r1, r3
D:\STM32\Program\1.11_Odchudzanie\um0427\FWLib\library\src/stm32f10x_tim.c:1322
   c:	8101      	strh	r1, [r0, #8]
D:\STM32\Program\1.11_Odchudzanie\um0427\FWLib\library\src/stm32f10x_tim.c:1323
   e:	4770      	bx	lr
Disassembly of section .text.TIM_ITRxExternalClockConfig:

00000000 <TIM_ITRxExternalClockConfig>:
TIM_ITRxExternalClockConfig():
D:\STM32\Program\1.11_Odchudzanie\um0427\FWLib\library\src/stm32f10x_tim.c:1039
   0:	b510      	push	{r4, lr}
   2:	4604      	mov	r4, r0
D:\STM32\Program\1.11_Odchudzanie\um0427\FWLib\library\src/stm32f10x_tim.c:1045
   4:	f7ff fffe 	bl	0 <TIM_ITRxExternalClockConfig>
D:\STM32\Program\1.11_Odchudzanie\um0427\FWLib\library\src/stm32f10x_tim.c:1048
   8:	8923      	ldrh	r3, [r4, #8]
   a:	b29b      	uxth	r3, r3
   c:	f043 0307 	orr.w	r3, r3, #7	; 0x7
  10:	8123      	strh	r3, [r4, #8]
D:\STM32\Program\1.11_Odchudzanie\um0427\FWLib\library\src/stm32f10x_tim.c:1049
  12:	bd10      	pop	{r4, pc}
Disassembly of section .text.TIM_EncoderInterfaceConfig:

00000000 <TIM_EncoderInterfaceConfig>:
TIM_EncoderInterfaceConfig():
D:\STM32\Program\1.11_Odchudzanie\um0427\FWLib\library\src/stm32f10x_tim.c:1351
   0:	b570      	push	{r4, r5, r6, lr}
D:\STM32\Program\1.11_Odchudzanie\um0427\FWLib\library\src/stm32f10x_tim.c:1363
   2:	8904      	ldrh	r4, [r0, #8]
D:\STM32\Program\1.11_Odchudzanie\um0427\FWLib\library\src/stm32f10x_tim.c:1366
   4:	8b05      	ldrh	r5, [r0, #24]
D:\STM32\Program\1.11_Odchudzanie\um0427\FWLib\library\src/stm32f10x_tim.c:1369
   6:	8c06      	ldrh	r6, [r0, #32]
D:\STM32\Program\1.11_Odchudzanie\um0427\FWLib\library\src/stm32f10x_tim.c:1376
   8:	f425 7540 	bic.w	r5, r5, #768	; 0x300
D:\STM32\Program\1.11_Odchudzanie\um0427\FWLib\library\src/stm32f10x_tim.c:1381
   c:	f026 0622 	bic.w	r6, r6, #34	; 0x22
D:\STM32\Program\1.11_Odchudzanie\um0427\FWLib\library\src/stm32f10x_tim.c:1376
  10:	f025 0503 	bic.w	r5, r5, #3	; 0x3
D:\STM32\Program\1.11_Odchudzanie\um0427\FWLib\library\src/stm32f10x_tim.c:1381
  14:	0436      	lsls	r6, r6, #16
D:\STM32\Program\1.11_Odchudzanie\um0427\FWLib\library\src/stm32f10x_tim.c:1372
  16:	f024 0407 	bic.w	r4, r4, #7	; 0x7
D:\STM32\Program\1.11_Odchudzanie\um0427\FWLib\library\src/stm32f10x_tim.c:1376
  1a:	042d      	lsls	r5, r5, #16
D:\STM32\Program\1.11_Odchudzanie\um0427\FWLib\library\src/stm32f10x_tim.c:1381
  1c:	0c36      	lsrs	r6, r6, #16
D:\STM32\Program\1.11_Odchudzanie\um0427\FWLib\library\src/stm32f10x_tim.c:1372
  1e:	0424      	lsls	r4, r4, #16
D:\STM32\Program\1.11_Odchudzanie\um0427\FWLib\library\src/stm32f10x_tim.c:1376
  20:	0c2d      	lsrs	r5, r5, #16
D:\STM32\Program\1.11_Odchudzanie\um0427\FWLib\library\src/stm32f10x_tim.c:1381
  22:	4332      	orrs	r2, r6
D:\STM32\Program\1.11_Odchudzanie\um0427\FWLib\library\src/stm32f10x_tim.c:1372
  24:	0c24      	lsrs	r4, r4, #16
D:\STM32\Program\1.11_Odchudzanie\um0427\FWLib\library\src/stm32f10x_tim.c:1377
  26:	f445 7580 	orr.w	r5, r5, #256	; 0x100
D:\STM32\Program\1.11_Odchudzanie\um0427\FWLib\library\src/stm32f10x_tim.c:1381
  2a:	ea42 1203 	orr.w	r2, r2, r3, lsl #4
D:\STM32\Program\1.11_Odchudzanie\um0427\FWLib\library\src/stm32f10x_tim.c:1373
  2e:	4321      	orrs	r1, r4
D:\STM32\Program\1.11_Odchudzanie\um0427\FWLib\library\src/stm32f10x_tim.c:1377
  30:	f045 0501 	orr.w	r5, r5, #1	; 0x1
D:\STM32\Program\1.11_Odchudzanie\um0427\FWLib\library\src/stm32f10x_tim.c:1381
  34:	b292      	uxth	r2, r2
D:\STM32\Program\1.11_Odchudzanie\um0427\FWLib\library\src/stm32f10x_tim.c:1384
  36:	8101      	strh	r1, [r0, #8]
D:\STM32\Program\1.11_Odchudzanie\um0427\FWLib\library\src/stm32f10x_tim.c:1387
  38:	8305      	strh	r5, [r0, #24]
D:\STM32\Program\1.11_Odchudzanie\um0427\FWLib\library\src/stm32f10x_tim.c:1390
  3a:	8402      	strh	r2, [r0, #32]
D:\STM32\Program\1.11_Odchudzanie\um0427\FWLib\library\src/stm32f10x_tim.c:1391
  3c:	bd70      	pop	{r4, r5, r6, pc}
  3e:	46c0      	nop			(mov r8, r8)
Disassembly of section .text.TIM_ForcedOC1Config:

00000000 <TIM_ForcedOC1Config>:
TIM_ForcedOC1Config():
D:\STM32\Program\1.11_Odchudzanie\um0427\FWLib\library\src/stm32f10x_tim.c:1415
   0:	8b03      	ldrh	r3, [r0, #24]
D:\STM32\Program\1.11_Odchudzanie\um0427\FWLib\library\src/stm32f10x_tim.c:1418
   2:	f023 0370 	bic.w	r3, r3, #112	; 0x70
   6:	041b      	lsls	r3, r3, #16
   8:	0c1b      	lsrs	r3, r3, #16
D:\STM32\Program\1.11_Odchudzanie\um0427\FWLib\library\src/stm32f10x_tim.c:1421
   a:	4319      	orrs	r1, r3
D:\STM32\Program\1.11_Odchudzanie\um0427\FWLib\library\src/stm32f10x_tim.c:1424
   c:	8301      	strh	r1, [r0, #24]
D:\STM32\Program\1.11_Odchudzanie\um0427\FWLib\library\src/stm32f10x_tim.c:1425
   e:	4770      	bx	lr
Disassembly of section .text.TIM_ForcedOC2Config:

00000000 <TIM_ForcedOC2Config>:
TIM_ForcedOC2Config():
D:\STM32\Program\1.11_Odchudzanie\um0427\FWLib\library\src/stm32f10x_tim.c:1442
   0:	8b03      	ldrh	r3, [r0, #24]
   2:	f423 43e0 	bic.w	r3, r3, #28672	; 0x7000
   6:	041b      	lsls	r3, r3, #16
   8:	0c1b      	lsrs	r3, r3, #16
D:\STM32\Program\1.11_Odchudzanie\um0427\FWLib\library\src/stm32f10x_tim.c:1455
   a:	ea43 2301 	orr.w	r3, r3, r1, lsl #8
   e:	b29b      	uxth	r3, r3
D:\STM32\Program\1.11_Odchudzanie\um0427\FWLib\library\src/stm32f10x_tim.c:1458
  10:	8303      	strh	r3, [r0, #24]
D:\STM32\Program\1.11_Odchudzanie\um0427\FWLib\library\src/stm32f10x_tim.c:1459
  12:	4770      	bx	lr
Disassembly of section .text.TIM_ForcedOC3Config:

00000000 <TIM_ForcedOC3Config>:
TIM_ForcedOC3Config():
D:\STM32\Program\1.11_Odchudzanie\um0427\FWLib\library\src/stm32f10x_tim.c:1476
   0:	8b83      	ldrh	r3, [r0, #28]
   2:	f023 0370 	bic.w	r3, r3, #112	; 0x70
   6:	041b      	lsls	r3, r3, #16
   8:	0c1b      	lsrs	r3, r3, #16
D:\STM32\Program\1.11_Odchudzanie\um0427\FWLib\library\src/stm32f10x_tim.c:1489
   a:	4319      	orrs	r1, r3
D:\STM32\Program\1.11_Odchudzanie\um0427\FWLib\library\src/stm32f10x_tim.c:1492
   c:	8381      	strh	r1, [r0, #28]
D:\STM32\Program\1.11_Odchudzanie\um0427\FWLib\library\src/stm32f10x_tim.c:1493
   e:	4770      	bx	lr
Disassembly of section .text.TIM_ForcedOC4Config:

00000000 <TIM_ForcedOC4Config>:
TIM_ForcedOC4Config():
D:\STM32\Program\1.11_Odchudzanie\um0427\FWLib\library\src/stm32f10x_tim.c:1510
   0:	8b83      	ldrh	r3, [r0, #28]
   2:	f423 43e0 	bic.w	r3, r3, #28672	; 0x7000
   6:	041b      	lsls	r3, r3, #16
   8:	0c1b      	lsrs	r3, r3, #16
D:\STM32\Program\1.11_Odchudzanie\um0427\FWLib\library\src/stm32f10x_tim.c:1522
   a:	ea43 2301 	orr.w	r3, r3, r1, lsl #8
   e:	b29b      	uxth	r3, r3
D:\STM32\Program\1.11_Odchudzanie\um0427\FWLib\library\src/stm32f10x_tim.c:1525
  10:	8383      	strh	r3, [r0, #28]
D:\STM32\Program\1.11_Odchudzanie\um0427\FWLib\library\src/stm32f10x_tim.c:1526
  12:	4770      	bx	lr
Disassembly of section .text.TIM_ARRPreloadConfig:

00000000 <TIM_ARRPreloadConfig>:
TIM_ARRPreloadConfig():
D:\STM32\Program\1.11_Odchudzanie\um0427\FWLib\library\src/stm32f10x_tim.c:1539
   0:	b121      	cbz	r1, c <TIM_ARRPreloadConfig+0xc>
D:\STM32\Program\1.11_Odchudzanie\um0427\FWLib\library\src/stm32f10x_tim.c:1547
   2:	8803      	ldrh	r3, [r0, #0]
   4:	b29b      	uxth	r3, r3
   6:	f043 0380 	orr.w	r3, r3, #128	; 0x80
   a:	e004      	b.n	16 <TIM_ARRPreloadConfig+0x16>
D:\STM32\Program\1.11_Odchudzanie\um0427\FWLib\library\src/stm32f10x_tim.c:1552
   c:	8803      	ldrh	r3, [r0, #0]
   e:	f023 0380 	bic.w	r3, r3, #128	; 0x80
  12:	059b      	lsls	r3, r3, #22
  14:	0d9b      	lsrs	r3, r3, #22
  16:	8003      	strh	r3, [r0, #0]
D:\STM32\Program\1.11_Odchudzanie\um0427\FWLib\library\src/stm32f10x_tim.c:1554
  18:	4770      	bx	lr
  1a:	46c0      	nop			(mov r8, r8)
Disassembly of section .text.TIM_SelectCOM:

00000000 <TIM_SelectCOM>:
TIM_SelectCOM():
D:\STM32\Program\1.11_Odchudzanie\um0427\FWLib\library\src/stm32f10x_tim.c:1566
   0:	b121      	cbz	r1, c <TIM_SelectCOM+0xc>
D:\STM32\Program\1.11_Odchudzanie\um0427\FWLib\library\src/stm32f10x_tim.c:1574
   2:	8883      	ldrh	r3, [r0, #4]
   4:	b29b      	uxth	r3, r3
   6:	f043 0304 	orr.w	r3, r3, #4	; 0x4
   a:	e004      	b.n	16 <TIM_SelectCOM+0x16>
D:\STM32\Program\1.11_Odchudzanie\um0427\FWLib\library\src/stm32f10x_tim.c:1579
   c:	8883      	ldrh	r3, [r0, #4]
   e:	f023 0304 	bic.w	r3, r3, #4	; 0x4
  12:	041b      	lsls	r3, r3, #16
  14:	0c1b      	lsrs	r3, r3, #16
  16:	8083      	strh	r3, [r0, #4]
D:\STM32\Program\1.11_Odchudzanie\um0427\FWLib\library\src/stm32f10x_tim.c:1581
  18:	4770      	bx	lr
  1a:	46c0      	nop			(mov r8, r8)
Disassembly of section .text.TIM_SelectCCDMA:

00000000 <TIM_SelectCCDMA>:
TIM_SelectCCDMA():
D:\STM32\Program\1.11_Odchudzanie\um0427\FWLib\library\src/stm32f10x_tim.c:1594
   0:	b121      	cbz	r1, c <TIM_SelectCCDMA+0xc>
D:\STM32\Program\1.11_Odchudzanie\um0427\FWLib\library\src/stm32f10x_tim.c:1602
   2:	8883      	ldrh	r3, [r0, #4]
   4:	b29b      	uxth	r3, r3
   6:	f043 0308 	orr.w	r3, r3, #8	; 0x8
   a:	e004      	b.n	16 <TIM_SelectCCDMA+0x16>
D:\STM32\Program\1.11_Odchudzanie\um0427\FWLib\library\src/stm32f10x_tim.c:1607
   c:	8883      	ldrh	r3, [r0, #4]
   e:	f023 0308 	bic.w	r3, r3, #8	; 0x8
  12:	041b      	lsls	r3, r3, #16
  14:	0c1b      	lsrs	r3, r3, #16
  16:	8083      	strh	r3, [r0, #4]
D:\STM32\Program\1.11_Odchudzanie\um0427\FWLib\library\src/stm32f10x_tim.c:1609
  18:	4770      	bx	lr
  1a:	46c0      	nop			(mov r8, r8)
Disassembly of section .text.TIM_CCPreloadControl:

00000000 <TIM_CCPreloadControl>:
TIM_CCPreloadControl():
D:\STM32\Program\1.11_Odchudzanie\um0427\FWLib\library\src/stm32f10x_tim.c:1622
   0:	b121      	cbz	r1, c <TIM_CCPreloadControl+0xc>
D:\STM32\Program\1.11_Odchudzanie\um0427\FWLib\library\src/stm32f10x_tim.c:1630
   2:	8883      	ldrh	r3, [r0, #4]
   4:	b29b      	uxth	r3, r3
   6:	f043 0301 	orr.w	r3, r3, #1	; 0x1
   a:	e004      	b.n	16 <TIM_CCPreloadControl+0x16>
D:\STM32\Program\1.11_Odchudzanie\um0427\FWLib\library\src/stm32f10x_tim.c:1635
   c:	8883      	ldrh	r3, [r0, #4]
   e:	f023 0301 	bic.w	r3, r3, #1	; 0x1
  12:	041b      	lsls	r3, r3, #16
  14:	0c1b      	lsrs	r3, r3, #16
  16:	8083      	strh	r3, [r0, #4]
D:\STM32\Program\1.11_Odchudzanie\um0427\FWLib\library\src/stm32f10x_tim.c:1637
  18:	4770      	bx	lr
  1a:	46c0      	nop			(mov r8, r8)
Disassembly of section .text.TIM_OC1PreloadConfig:

00000000 <TIM_OC1PreloadConfig>:
TIM_OC1PreloadConfig():
D:\STM32\Program\1.11_Odchudzanie\um0427\FWLib\library\src/stm32f10x_tim.c:1653
   0:	8b03      	ldrh	r3, [r0, #24]
   2:	f023 0308 	bic.w	r3, r3, #8	; 0x8
   6:	041b      	lsls	r3, r3, #16
   8:	0c1b      	lsrs	r3, r3, #16
D:\STM32\Program\1.11_Odchudzanie\um0427\FWLib\library\src/stm32f10x_tim.c:1666
   a:	4319      	orrs	r1, r3
D:\STM32\Program\1.11_Odchudzanie\um0427\FWLib\library\src/stm32f10x_tim.c:1669
   c:	8301      	strh	r1, [r0, #24]
D:\STM32\Program\1.11_Odchudzanie\um0427\FWLib\library\src/stm32f10x_tim.c:1670
   e:	4770      	bx	lr
Disassembly of section .text.TIM_OC2PreloadConfig:

00000000 <TIM_OC2PreloadConfig>:
TIM_OC2PreloadConfig():
D:\STM32\Program\1.11_Odchudzanie\um0427\FWLib\library\src/stm32f10x_tim.c:1686
   0:	8b03      	ldrh	r3, [r0, #24]
   2:	f423 6300 	bic.w	r3, r3, #2048	; 0x800
   6:	041b      	lsls	r3, r3, #16
   8:	0c1b      	lsrs	r3, r3, #16
D:\STM32\Program\1.11_Odchudzanie\um0427\FWLib\library\src/stm32f10x_tim.c:1699
   a:	ea43 2301 	orr.w	r3, r3, r1, lsl #8
   e:	b29b      	uxth	r3, r3
D:\STM32\Program\1.11_Odchudzanie\um0427\FWLib\library\src/stm32f10x_tim.c:1702
  10:	8303      	strh	r3, [r0, #24]
D:\STM32\Program\1.11_Odchudzanie\um0427\FWLib\library\src/stm32f10x_tim.c:1703
  12:	4770      	bx	lr
Disassembly of section .text.TIM_OC3PreloadConfig:

00000000 <TIM_OC3PreloadConfig>:
TIM_OC3PreloadConfig():
D:\STM32\Program\1.11_Odchudzanie\um0427\FWLib\library\src/stm32f10x_tim.c:1719
   0:	8b83      	ldrh	r3, [r0, #28]
   2:	f023 0308 	bic.w	r3, r3, #8	; 0x8
   6:	041b      	lsls	r3, r3, #16
   8:	0c1b      	lsrs	r3, r3, #16
D:\STM32\Program\1.11_Odchudzanie\um0427\FWLib\library\src/stm32f10x_tim.c:1732
   a:	4319      	orrs	r1, r3
D:\STM32\Program\1.11_Odchudzanie\um0427\FWLib\library\src/stm32f10x_tim.c:1735
   c:	8381      	strh	r1, [r0, #28]
D:\STM32\Program\1.11_Odchudzanie\um0427\FWLib\library\src/stm32f10x_tim.c:1736
   e:	4770      	bx	lr
Disassembly of section .text.TIM_OC4PreloadConfig:

00000000 <TIM_OC4PreloadConfig>:
TIM_OC4PreloadConfig():
D:\STM32\Program\1.11_Odchudzanie\um0427\FWLib\library\src/stm32f10x_tim.c:1752
   0:	8b83      	ldrh	r3, [r0, #28]
   2:	f423 6300 	bic.w	r3, r3, #2048	; 0x800
   6:	041b      	lsls	r3, r3, #16
   8:	0c1b      	lsrs	r3, r3, #16
D:\STM32\Program\1.11_Odchudzanie\um0427\FWLib\library\src/stm32f10x_tim.c:1765
   a:	ea43 2301 	orr.w	r3, r3, r1, lsl #8
   e:	b29b      	uxth	r3, r3
D:\STM32\Program\1.11_Odchudzanie\um0427\FWLib\library\src/stm32f10x_tim.c:1768
  10:	8383      	strh	r3, [r0, #28]
D:\STM32\Program\1.11_Odchudzanie\um0427\FWLib\library\src/stm32f10x_tim.c:1769
  12:	4770      	bx	lr
Disassembly of section .text.TIM_OC1FastConfig:

00000000 <TIM_OC1FastConfig>:
TIM_OC1FastConfig():
D:\STM32\Program\1.11_Odchudzanie\um0427\FWLib\library\src/stm32f10x_tim.c:1784
   0:	8b03      	ldrh	r3, [r0, #24]
   2:	f023 0304 	bic.w	r3, r3, #4	; 0x4
   6:	041b      	lsls	r3, r3, #16
   8:	0c1b      	lsrs	r3, r3, #16
D:\STM32\Program\1.11_Odchudzanie\um0427\FWLib\library\src/stm32f10x_tim.c:1798
   a:	4319      	orrs	r1, r3
D:\STM32\Program\1.11_Odchudzanie\um0427\FWLib\library\src/stm32f10x_tim.c:1801
   c:	8301      	strh	r1, [r0, #24]
D:\STM32\Program\1.11_Odchudzanie\um0427\FWLib\library\src/stm32f10x_tim.c:1802
   e:	4770      	bx	lr
Disassembly of section .text.TIM_OC2FastConfig:

00000000 <TIM_OC2FastConfig>:
TIM_OC2FastConfig():
D:\STM32\Program\1.11_Odchudzanie\um0427\FWLib\library\src/stm32f10x_tim.c:1817
   0:	8b03      	ldrh	r3, [r0, #24]
   2:	f423 6380 	bic.w	r3, r3, #1024	; 0x400
   6:	041b      	lsls	r3, r3, #16
   8:	0c1b      	lsrs	r3, r3, #16
D:\STM32\Program\1.11_Odchudzanie\um0427\FWLib\library\src/stm32f10x_tim.c:1831
   a:	ea43 2301 	orr.w	r3, r3, r1, lsl #8
   e:	b29b      	uxth	r3, r3
D:\STM32\Program\1.11_Odchudzanie\um0427\FWLib\library\src/stm32f10x_tim.c:1834
  10:	8303      	strh	r3, [r0, #24]
D:\STM32\Program\1.11_Odchudzanie\um0427\FWLib\library\src/stm32f10x_tim.c:1835
  12:	4770      	bx	lr
Disassembly of section .text.TIM_OC3FastConfig:

00000000 <TIM_OC3FastConfig>:
TIM_OC3FastConfig():
D:\STM32\Program\1.11_Odchudzanie\um0427\FWLib\library\src/stm32f10x_tim.c:1850
   0:	8b83      	ldrh	r3, [r0, #28]
   2:	f023 0304 	bic.w	r3, r3, #4	; 0x4
   6:	041b      	lsls	r3, r3, #16
   8:	0c1b      	lsrs	r3, r3, #16
D:\STM32\Program\1.11_Odchudzanie\um0427\FWLib\library\src/stm32f10x_tim.c:1864
   a:	4319      	orrs	r1, r3
D:\STM32\Program\1.11_Odchudzanie\um0427\FWLib\library\src/stm32f10x_tim.c:1867
   c:	8381      	strh	r1, [r0, #28]
D:\STM32\Program\1.11_Odchudzanie\um0427\FWLib\library\src/stm32f10x_tim.c:1868
   e:	4770      	bx	lr
Disassembly of section .text.TIM_OC4FastConfig:

00000000 <TIM_OC4FastConfig>:
TIM_OC4FastConfig():
D:\STM32\Program\1.11_Odchudzanie\um0427\FWLib\library\src/stm32f10x_tim.c:1883
   0:	8b83      	ldrh	r3, [r0, #28]
   2:	f423 6380 	bic.w	r3, r3, #1024	; 0x400
   6:	041b      	lsls	r3, r3, #16
   8:	0c1b      	lsrs	r3, r3, #16
D:\STM32\Program\1.11_Odchudzanie\um0427\FWLib\library\src/stm32f10x_tim.c:1897
   a:	ea43 2301 	orr.w	r3, r3, r1, lsl #8
   e:	b29b      	uxth	r3, r3
D:\STM32\Program\1.11_Odchudzanie\um0427\FWLib\library\src/stm32f10x_tim.c:1900
  10:	8383      	strh	r3, [r0, #28]
D:\STM32\Program\1.11_Odchudzanie\um0427\FWLib\library\src/stm32f10x_tim.c:1901
  12:	4770      	bx	lr
Disassembly of section .text.TIM_ClearOC1Ref:

00000000 <TIM_ClearOC1Ref>:
TIM_ClearOC1Ref():
D:\STM32\Program\1.11_Odchudzanie\um0427\FWLib\library\src/stm32f10x_tim.c:1916
   0:	8b03      	ldrh	r3, [r0, #24]
   2:	f023 0380 	bic.w	r3, r3, #128	; 0x80
   6:	041b      	lsls	r3, r3, #16
   8:	0c1b      	lsrs	r3, r3, #16
D:\STM32\Program\1.11_Odchudzanie\um0427\FWLib\library\src/stm32f10x_tim.c:1929
   a:	4319      	orrs	r1, r3
D:\STM32\Program\1.11_Odchudzanie\um0427\FWLib\library\src/stm32f10x_tim.c:1932
   c:	8301      	strh	r1, [r0, #24]
D:\STM32\Program\1.11_Odchudzanie\um0427\FWLib\library\src/stm32f10x_tim.c:1933
   e:	4770      	bx	lr
Disassembly of section .text.TIM_ClearOC2Ref:

00000000 <TIM_ClearOC2Ref>:
TIM_ClearOC2Ref():
D:\STM32\Program\1.11_Odchudzanie\um0427\FWLib\library\src/stm32f10x_tim.c:1948
   0:	8b03      	ldrh	r3, [r0, #24]
   2:	045b      	lsls	r3, r3, #17
   4:	0c5b      	lsrs	r3, r3, #17
D:\STM32\Program\1.11_Odchudzanie\um0427\FWLib\library\src/stm32f10x_tim.c:1961
   6:	ea43 2301 	orr.w	r3, r3, r1, lsl #8
   a:	b29b      	uxth	r3, r3
D:\STM32\Program\1.11_Odchudzanie\um0427\FWLib\library\src/stm32f10x_tim.c:1964
   c:	8303      	strh	r3, [r0, #24]
D:\STM32\Program\1.11_Odchudzanie\um0427\FWLib\library\src/stm32f10x_tim.c:1965
   e:	4770      	bx	lr
Disassembly of section .text.TIM_ClearOC3Ref:

00000000 <TIM_ClearOC3Ref>:
TIM_ClearOC3Ref():
D:\STM32\Program\1.11_Odchudzanie\um0427\FWLib\library\src/stm32f10x_tim.c:1980
   0:	8b83      	ldrh	r3, [r0, #28]
   2:	f023 0380 	bic.w	r3, r3, #128	; 0x80
   6:	041b      	lsls	r3, r3, #16
   8:	0c1b      	lsrs	r3, r3, #16
D:\STM32\Program\1.11_Odchudzanie\um0427\FWLib\library\src/stm32f10x_tim.c:1993
   a:	4319      	orrs	r1, r3
D:\STM32\Program\1.11_Odchudzanie\um0427\FWLib\library\src/stm32f10x_tim.c:1996
   c:	8381      	strh	r1, [r0, #28]
D:\STM32\Program\1.11_Odchudzanie\um0427\FWLib\library\src/stm32f10x_tim.c:1997
   e:	4770      	bx	lr
Disassembly of section .text.TIM_ClearOC4Ref:

00000000 <TIM_ClearOC4Ref>:
TIM_ClearOC4Ref():
D:\STM32\Program\1.11_Odchudzanie\um0427\FWLib\library\src/stm32f10x_tim.c:2012
   0:	8b83      	ldrh	r3, [r0, #28]
   2:	045b      	lsls	r3, r3, #17
   4:	0c5b      	lsrs	r3, r3, #17
D:\STM32\Program\1.11_Odchudzanie\um0427\FWLib\library\src/stm32f10x_tim.c:2025
   6:	ea43 2301 	orr.w	r3, r3, r1, lsl #8
   a:	b29b      	uxth	r3, r3
D:\STM32\Program\1.11_Odchudzanie\um0427\FWLib\library\src/stm32f10x_tim.c:2028
   c:	8383      	strh	r3, [r0, #28]
D:\STM32\Program\1.11_Odchudzanie\um0427\FWLib\library\src/stm32f10x_tim.c:2029
   e:	4770      	bx	lr
Disassembly of section .text.TIM_OC1PolarityConfig:

00000000 <TIM_OC1PolarityConfig>:
TIM_OC1PolarityConfig():
D:\STM32\Program\1.11_Odchudzanie\um0427\FWLib\library\src/stm32f10x_tim.c:2044
   0:	8c03      	ldrh	r3, [r0, #32]
   2:	f023 0302 	bic.w	r3, r3, #2	; 0x2
   6:	041b      	lsls	r3, r3, #16
   8:	0c1b      	lsrs	r3, r3, #16
D:\STM32\Program\1.11_Odchudzanie\um0427\FWLib\library\src/stm32f10x_tim.c:2055
   a:	4319      	orrs	r1, r3
D:\STM32\Program\1.11_Odchudzanie\um0427\FWLib\library\src/stm32f10x_tim.c:2058
   c:	8401      	strh	r1, [r0, #32]
D:\STM32\Program\1.11_Odchudzanie\um0427\FWLib\library\src/stm32f10x_tim.c:2059
   e:	4770      	bx	lr
Disassembly of section .text.TIM_OC1NPolarityConfig:

00000000 <TIM_OC1NPolarityConfig>:
TIM_OC1NPolarityConfig():
D:\STM32\Program\1.11_Odchudzanie\um0427\FWLib\library\src/stm32f10x_tim.c:2073
   0:	8c03      	ldrh	r3, [r0, #32]
   2:	f023 0308 	bic.w	r3, r3, #8	; 0x8
   6:	041b      	lsls	r3, r3, #16
   8:	0c1b      	lsrs	r3, r3, #16
D:\STM32\Program\1.11_Odchudzanie\um0427\FWLib\library\src/stm32f10x_tim.c:2084
   a:	4319      	orrs	r1, r3
D:\STM32\Program\1.11_Odchudzanie\um0427\FWLib\library\src/stm32f10x_tim.c:2087
   c:	8401      	strh	r1, [r0, #32]
D:\STM32\Program\1.11_Odchudzanie\um0427\FWLib\library\src/stm32f10x_tim.c:2088
   e:	4770      	bx	lr
Disassembly of section .text.TIM_OC2PolarityConfig:

00000000 <TIM_OC2PolarityConfig>:
TIM_OC2PolarityConfig():
D:\STM32\Program\1.11_Odchudzanie\um0427\FWLib\library\src/stm32f10x_tim.c:2103
   0:	8c03      	ldrh	r3, [r0, #32]
   2:	f023 0320 	bic.w	r3, r3, #32	; 0x20
   6:	041b      	lsls	r3, r3, #16
   8:	0c1b      	lsrs	r3, r3, #16
D:\STM32\Program\1.11_Odchudzanie\um0427\FWLib\library\src/stm32f10x_tim.c:2114
   a:	ea43 1301 	orr.w	r3, r3, r1, lsl #4
   e:	b29b      	uxth	r3, r3
D:\STM32\Program\1.11_Odchudzanie\um0427\FWLib\library\src/stm32f10x_tim.c:2117
  10:	8403      	strh	r3, [r0, #32]
D:\STM32\Program\1.11_Odchudzanie\um0427\FWLib\library\src/stm32f10x_tim.c:2118
  12:	4770      	bx	lr
Disassembly of section .text.TIM_OC2NPolarityConfig:

00000000 <TIM_OC2NPolarityConfig>:
TIM_OC2NPolarityConfig():
D:\STM32\Program\1.11_Odchudzanie\um0427\FWLib\library\src/stm32f10x_tim.c:2132
   0:	8c03      	ldrh	r3, [r0, #32]
   2:	f023 0380 	bic.w	r3, r3, #128	; 0x80
   6:	041b      	lsls	r3, r3, #16
   8:	0c1b      	lsrs	r3, r3, #16
D:\STM32\Program\1.11_Odchudzanie\um0427\FWLib\library\src/stm32f10x_tim.c:2143
   a:	ea43 1301 	orr.w	r3, r3, r1, lsl #4
   e:	b29b      	uxth	r3, r3
D:\STM32\Program\1.11_Odchudzanie\um0427\FWLib\library\src/stm32f10x_tim.c:2146
  10:	8403      	strh	r3, [r0, #32]
D:\STM32\Program\1.11_Odchudzanie\um0427\FWLib\library\src/stm32f10x_tim.c:2147
  12:	4770      	bx	lr
Disassembly of section .text.TIM_OC3PolarityConfig:

00000000 <TIM_OC3PolarityConfig>:
TIM_OC3PolarityConfig():
D:\STM32\Program\1.11_Odchudzanie\um0427\FWLib\library\src/stm32f10x_tim.c:2162
   0:	8c03      	ldrh	r3, [r0, #32]
   2:	f423 7300 	bic.w	r3, r3, #512	; 0x200
   6:	041b      	lsls	r3, r3, #16
   8:	0c1b      	lsrs	r3, r3, #16
D:\STM32\Program\1.11_Odchudzanie\um0427\FWLib\library\src/stm32f10x_tim.c:2173
   a:	ea43 2301 	orr.w	r3, r3, r1, lsl #8
   e:	b29b      	uxth	r3, r3
D:\STM32\Program\1.11_Odchudzanie\um0427\FWLib\library\src/stm32f10x_tim.c:2176
  10:	8403      	strh	r3, [r0, #32]
D:\STM32\Program\1.11_Odchudzanie\um0427\FWLib\library\src/stm32f10x_tim.c:2177
  12:	4770      	bx	lr
Disassembly of section .text.TIM_OC3NPolarityConfig:

00000000 <TIM_OC3NPolarityConfig>:
TIM_OC3NPolarityConfig():
D:\STM32\Program\1.11_Odchudzanie\um0427\FWLib\library\src/stm32f10x_tim.c:2191
   0:	8c03      	ldrh	r3, [r0, #32]
   2:	f423 6300 	bic.w	r3, r3, #2048	; 0x800
   6:	041b      	lsls	r3, r3, #16
   8:	0c1b      	lsrs	r3, r3, #16
D:\STM32\Program\1.11_Odchudzanie\um0427\FWLib\library\src/stm32f10x_tim.c:2202
   a:	ea43 2301 	orr.w	r3, r3, r1, lsl #8
   e:	b29b      	uxth	r3, r3
D:\STM32\Program\1.11_Odchudzanie\um0427\FWLib\library\src/stm32f10x_tim.c:2205
  10:	8403      	strh	r3, [r0, #32]
D:\STM32\Program\1.11_Odchudzanie\um0427\FWLib\library\src/stm32f10x_tim.c:2206
  12:	4770      	bx	lr
Disassembly of section .text.TIM_OC4PolarityConfig:

00000000 <TIM_OC4PolarityConfig>:
TIM_OC4PolarityConfig():
D:\STM32\Program\1.11_Odchudzanie\um0427\FWLib\library\src/stm32f10x_tim.c:2228
   0:	8c03      	ldrh	r3, [r0, #32]
D:\STM32\Program\1.11_Odchudzanie\um0427\FWLib\library\src/stm32f10x_tim.c:2231
   2:	f423 5300 	bic.w	r3, r3, #8192	; 0x2000
   6:	041b      	lsls	r3, r3, #16
   8:	0c1b      	lsrs	r3, r3, #16
D:\STM32\Program\1.11_Odchudzanie\um0427\FWLib\library\src/stm32f10x_tim.c:2232
   a:	ea43 3301 	orr.w	r3, r3, r1, lsl #12
   e:	b29b      	uxth	r3, r3
D:\STM32\Program\1.11_Odchudzanie\um0427\FWLib\library\src/stm32f10x_tim.c:2235
  10:	8403      	strh	r3, [r0, #32]
D:\STM32\Program\1.11_Odchudzanie\um0427\FWLib\library\src/stm32f10x_tim.c:2236
  12:	4770      	bx	lr
Disassembly of section .text.TIM_CCxCmd:

00000000 <TIM_CCxCmd>:
TIM_CCxCmd():
D:\STM32\Program\1.11_Odchudzanie\um0427\FWLib\library\src/stm32f10x_tim.c:2255
   0:	2301      	movs	r3, #1
   2:	408b      	lsls	r3, r1
D:\STM32\Program\1.11_Odchudzanie\um0427\FWLib\library\src/stm32f10x_tim.c:2265
   4:	408a      	lsls	r2, r1
D:\STM32\Program\1.11_Odchudzanie\um0427\FWLib\library\src/stm32f10x_tim.c:2255
   6:	b510      	push	{r4, lr}
D:\STM32\Program\1.11_Odchudzanie\um0427\FWLib\library\src/stm32f10x_tim.c:2262
   8:	8c04      	ldrh	r4, [r0, #32]
   a:	b2a4      	uxth	r4, r4
   c:	ea24 0403 	bic.w	r4, r4, r3
  10:	8404      	strh	r4, [r0, #32]
D:\STM32\Program\1.11_Odchudzanie\um0427\FWLib\library\src/stm32f10x_tim.c:2265
  12:	8c03      	ldrh	r3, [r0, #32]
  14:	431a      	orrs	r2, r3
  16:	b292      	uxth	r2, r2
  18:	8402      	strh	r2, [r0, #32]
D:\STM32\Program\1.11_Odchudzanie\um0427\FWLib\library\src/stm32f10x_tim.c:2266
  1a:	bd10      	pop	{r4, pc}
Disassembly of section .text.TIM_CCxNCmd:

00000000 <TIM_CCxNCmd>:
TIM_CCxNCmd():
D:\STM32\Program\1.11_Odchudzanie\um0427\FWLib\library\src/stm32f10x_tim.c:2283
   0:	2304      	movs	r3, #4
   2:	408b      	lsls	r3, r1
D:\STM32\Program\1.11_Odchudzanie\um0427\FWLib\library\src/stm32f10x_tim.c:2293
   4:	408a      	lsls	r2, r1
D:\STM32\Program\1.11_Odchudzanie\um0427\FWLib\library\src/stm32f10x_tim.c:2283
   6:	b510      	push	{r4, lr}
D:\STM32\Program\1.11_Odchudzanie\um0427\FWLib\library\src/stm32f10x_tim.c:2290
   8:	8c04      	ldrh	r4, [r0, #32]
   a:	b2a4      	uxth	r4, r4
   c:	ea24 0403 	bic.w	r4, r4, r3
  10:	8404      	strh	r4, [r0, #32]
D:\STM32\Program\1.11_Odchudzanie\um0427\FWLib\library\src/stm32f10x_tim.c:2293
  12:	8c03      	ldrh	r3, [r0, #32]
  14:	431a      	orrs	r2, r3
  16:	b292      	uxth	r2, r2
  18:	8402      	strh	r2, [r0, #32]
D:\STM32\Program\1.11_Odchudzanie\um0427\FWLib\library\src/stm32f10x_tim.c:2294
  1a:	bd10      	pop	{r4, pc}
Disassembly of section .text.TIM_SelectOCxM:

00000000 <TIM_SelectOCxM>:
TIM_SelectOCxM():
D:\STM32\Program\1.11_Odchudzanie\um0427\FWLib\library\src/stm32f10x_tim.c:2323
   0:	2301      	movs	r3, #1
   2:	408b      	lsls	r3, r1
   4:	b513      	push	{r0, r1, r4, lr}
   6:	4614      	mov	r4, r2
D:\STM32\Program\1.11_Odchudzanie\um0427\FWLib\library\src/stm32f10x_tim.c:2330
   8:	8c02      	ldrh	r2, [r0, #32]
D:\STM32\Program\1.11_Odchudzanie\um0427\FWLib\library\src/stm32f10x_tim.c:2323
   a:	9001      	str	r0, [sp, #4]
D:\STM32\Program\1.11_Odchudzanie\um0427\FWLib\library\src/stm32f10x_tim.c:2330
   c:	b292      	uxth	r2, r2
   e:	ea22 0203 	bic.w	r2, r2, r3
  12:	8402      	strh	r2, [r0, #32]
D:\STM32\Program\1.11_Odchudzanie\um0427\FWLib\library\src/stm32f10x_tim.c:2332
  14:	b109      	cbz	r1, 1a <TIM_SelectOCxM+0x1a>
  16:	2908      	cmp	r1, #8
  18:	d10a      	bne.n	30 <TIM_SelectOCxM+0x30>
D:\STM32\Program\1.11_Odchudzanie\um0427\FWLib\library\src/stm32f10x_tim.c:2335
  1a:	0849      	lsrs	r1, r1, #1
  1c:	f100 0218 	add.w	r2, r0, #24	; 0x18
  20:	5850      	ldr	r0, [r2, r1]
  22:	f64f 738f 	movw	r3, #65423	; 0xff8f
  26:	ea00 0303 	and.w	r3, r0, r3
  2a:	5053      	str	r3, [r2, r1]
D:\STM32\Program\1.11_Odchudzanie\um0427\FWLib\library\src/stm32f10x_tim.c:2338
  2c:	5054      	str	r4, [r2, r1]
D:\STM32\Program\1.11_Odchudzanie\um0427\FWLib\library\src/stm32f10x_tim.c:2332
  2e:	e00d      	b.n	4c <TIM_SelectOCxM+0x4c>
D:\STM32\Program\1.11_Odchudzanie\um0427\FWLib\library\src/stm32f10x_tim.c:2344
  30:	1f0a      	subs	r2, r1, #4
  32:	f3c2 024e 	ubfx	r2, r2, #1, #15
  36:	f100 0118 	add.w	r1, r0, #24	; 0x18
  3a:	5888      	ldr	r0, [r1, r2]
  3c:	f648 73ff 	movw	r3, #36863	; 0x8fff
  40:	ea00 0303 	and.w	r3, r0, r3
  44:	508b      	str	r3, [r1, r2]
D:\STM32\Program\1.11_Odchudzanie\um0427\FWLib\library\src/stm32f10x_tim.c:2347
  46:	0223      	lsls	r3, r4, #8
  48:	b29b      	uxth	r3, r3
  4a:	508b      	str	r3, [r1, r2]
D:\STM32\Program\1.11_Odchudzanie\um0427\FWLib\library\src/stm32f10x_tim.c:2349
  4c:	bd1c      	pop	{r2, r3, r4, pc}
  4e:	46c0      	nop			(mov r8, r8)
Disassembly of section .text.TIM_UpdateDisableConfig:

00000000 <TIM_UpdateDisableConfig>:
TIM_UpdateDisableConfig():
D:\STM32\Program\1.11_Odchudzanie\um0427\FWLib\library\src/stm32f10x_tim.c:2361
   0:	b121      	cbz	r1, c <TIM_UpdateDisableConfig+0xc>
D:\STM32\Program\1.11_Odchudzanie\um0427\FWLib\library\src/stm32f10x_tim.c:2369
   2:	8803      	ldrh	r3, [r0, #0]
   4:	b29b      	uxth	r3, r3
   6:	f043 0302 	orr.w	r3, r3, #2	; 0x2
   a:	e004      	b.n	16 <TIM_UpdateDisableConfig+0x16>
D:\STM32\Program\1.11_Odchudzanie\um0427\FWLib\library\src/stm32f10x_tim.c:2374
   c:	8803      	ldrh	r3, [r0, #0]
   e:	f023 0302 	bic.w	r3, r3, #2	; 0x2
  12:	059b      	lsls	r3, r3, #22
  14:	0d9b      	lsrs	r3, r3, #22
  16:	8003      	strh	r3, [r0, #0]
D:\STM32\Program\1.11_Odchudzanie\um0427\FWLib\library\src/stm32f10x_tim.c:2376
  18:	4770      	bx	lr
  1a:	46c0      	nop			(mov r8, r8)
Disassembly of section .text.TIM_UpdateRequestConfig:

00000000 <TIM_UpdateRequestConfig>:
TIM_UpdateRequestConfig():
D:\STM32\Program\1.11_Odchudzanie\um0427\FWLib\library\src/stm32f10x_tim.c:2395
   0:	b121      	cbz	r1, c <TIM_UpdateRequestConfig+0xc>
D:\STM32\Program\1.11_Odchudzanie\um0427\FWLib\library\src/stm32f10x_tim.c:2398
   2:	8803      	ldrh	r3, [r0, #0]
   4:	b29b      	uxth	r3, r3
   6:	f043 0304 	orr.w	r3, r3, #4	; 0x4
   a:	e004      	b.n	16 <TIM_UpdateRequestConfig+0x16>
D:\STM32\Program\1.11_Odchudzanie\um0427\FWLib\library\src/stm32f10x_tim.c:2403
   c:	8803      	ldrh	r3, [r0, #0]
   e:	f023 0304 	bic.w	r3, r3, #4	; 0x4
  12:	059b      	lsls	r3, r3, #22
  14:	0d9b      	lsrs	r3, r3, #22
  16:	8003      	strh	r3, [r0, #0]
D:\STM32\Program\1.11_Odchudzanie\um0427\FWLib\library\src/stm32f10x_tim.c:2405
  18:	4770      	bx	lr
  1a:	46c0      	nop			(mov r8, r8)
Disassembly of section .text.TIM_SelectHallSensor:

00000000 <TIM_SelectHallSensor>:
TIM_SelectHallSensor():
D:\STM32\Program\1.11_Odchudzanie\um0427\FWLib\library\src/stm32f10x_tim.c:2417
   0:	b121      	cbz	r1, c <TIM_SelectHallSensor+0xc>
D:\STM32\Program\1.11_Odchudzanie\um0427\FWLib\library\src/stm32f10x_tim.c:2425
   2:	8883      	ldrh	r3, [r0, #4]
   4:	b29b      	uxth	r3, r3
   6:	f043 0380 	orr.w	r3, r3, #128	; 0x80
   a:	e004      	b.n	16 <TIM_SelectHallSensor+0x16>
D:\STM32\Program\1.11_Odchudzanie\um0427\FWLib\library\src/stm32f10x_tim.c:2430
   c:	8883      	ldrh	r3, [r0, #4]
   e:	f023 0380 	bic.w	r3, r3, #128	; 0x80
  12:	041b      	lsls	r3, r3, #16
  14:	0c1b      	lsrs	r3, r3, #16
  16:	8083      	strh	r3, [r0, #4]
D:\STM32\Program\1.11_Odchudzanie\um0427\FWLib\library\src/stm32f10x_tim.c:2432
  18:	4770      	bx	lr
  1a:	46c0      	nop			(mov r8, r8)
Disassembly of section .text.TIM_SelectOnePulseMode:

00000000 <TIM_SelectOnePulseMode>:
TIM_SelectOnePulseMode():
D:\STM32\Program\1.11_Odchudzanie\um0427\FWLib\library\src/stm32f10x_tim.c:2446
   0:	8803      	ldrh	r3, [r0, #0]
   2:	f023 0308 	bic.w	r3, r3, #8	; 0x8
   6:	059b      	lsls	r3, r3, #22
   8:	0d9b      	lsrs	r3, r3, #22
   a:	8003      	strh	r3, [r0, #0]
D:\STM32\Program\1.11_Odchudzanie\um0427\FWLib\library\src/stm32f10x_tim.c:2455
   c:	8803      	ldrh	r3, [r0, #0]
   e:	b29b      	uxth	r3, r3
  10:	4319      	orrs	r1, r3
  12:	8001      	strh	r1, [r0, #0]
D:\STM32\Program\1.11_Odchudzanie\um0427\FWLib\library\src/stm32f10x_tim.c:2456
  14:	4770      	bx	lr
  16:	46c0      	nop			(mov r8, r8)
Disassembly of section .text.TIM_SelectOutputTrigger:

00000000 <TIM_SelectOutputTrigger>:
TIM_SelectOutputTrigger():
D:\STM32\Program\1.11_Odchudzanie\um0427\FWLib\library\src/stm32f10x_tim.c:2479
   0:	8883      	ldrh	r3, [r0, #4]
   2:	f023 0370 	bic.w	r3, r3, #112	; 0x70
   6:	041b      	lsls	r3, r3, #16
   8:	0c1b      	lsrs	r3, r3, #16
   a:	8083      	strh	r3, [r0, #4]
D:\STM32\Program\1.11_Odchudzanie\um0427\FWLib\library\src/stm32f10x_tim.c:2489
   c:	8883      	ldrh	r3, [r0, #4]
   e:	b29b      	uxth	r3, r3
  10:	4319      	orrs	r1, r3
  12:	8081      	strh	r1, [r0, #4]
D:\STM32\Program\1.11_Odchudzanie\um0427\FWLib\library\src/stm32f10x_tim.c:2490
  14:	4770      	bx	lr
  16:	46c0      	nop			(mov r8, r8)
Disassembly of section .text.TIM_SelectSlaveMode:

00000000 <TIM_SelectSlaveMode>:
TIM_SelectSlaveMode():
D:\STM32\Program\1.11_Odchudzanie\um0427\FWLib\library\src/stm32f10x_tim.c:2507
   0:	8903      	ldrh	r3, [r0, #8]
   2:	f023 0307 	bic.w	r3, r3, #7	; 0x7
   6:	041b      	lsls	r3, r3, #16
   8:	0c1b      	lsrs	r3, r3, #16
   a:	8103      	strh	r3, [r0, #8]
D:\STM32\Program\1.11_Odchudzanie\um0427\FWLib\library\src/stm32f10x_tim.c:2516
   c:	8903      	ldrh	r3, [r0, #8]
   e:	b29b      	uxth	r3, r3
  10:	4319      	orrs	r1, r3
  12:	8101      	strh	r1, [r0, #8]
D:\STM32\Program\1.11_Odchudzanie\um0427\FWLib\library\src/stm32f10x_tim.c:2517
  14:	4770      	bx	lr
  16:	46c0      	nop			(mov r8, r8)
Disassembly of section .text.TIM_SelectMasterSlaveMode:

00000000 <TIM_SelectMasterSlaveMode>:
TIM_SelectMasterSlaveMode():
D:\STM32\Program\1.11_Odchudzanie\um0427\FWLib\library\src/stm32f10x_tim.c:2533
   0:	8903      	ldrh	r3, [r0, #8]
   2:	f023 0380 	bic.w	r3, r3, #128	; 0x80
   6:	041b      	lsls	r3, r3, #16
   8:	0c1b      	lsrs	r3, r3, #16
   a:	8103      	strh	r3, [r0, #8]
D:\STM32\Program\1.11_Odchudzanie\um0427\FWLib\library\src/stm32f10x_tim.c:2542
   c:	8903      	ldrh	r3, [r0, #8]
   e:	b29b      	uxth	r3, r3
  10:	4319      	orrs	r1, r3
  12:	8101      	strh	r1, [r0, #8]
D:\STM32\Program\1.11_Odchudzanie\um0427\FWLib\library\src/stm32f10x_tim.c:2543
  14:	4770      	bx	lr
  16:	46c0      	nop			(mov r8, r8)
Disassembly of section .text.TIM_SetCounter:

00000000 <TIM_SetCounter>:
TIM_SetCounter():
D:\STM32\Program\1.11_Odchudzanie\um0427\FWLib\library\src/stm32f10x_tim.c:2554
   0:	8481      	strh	r1, [r0, #36]
D:\STM32\Program\1.11_Odchudzanie\um0427\FWLib\library\src/stm32f10x_tim.c:2560
   2:	4770      	bx	lr
Disassembly of section .text.TIM_SetAutoreload:

00000000 <TIM_SetAutoreload>:
TIM_SetAutoreload():
D:\STM32\Program\1.11_Odchudzanie\um0427\FWLib\library\src/stm32f10x_tim.c:2571
   0:	8581      	strh	r1, [r0, #44]
D:\STM32\Program\1.11_Odchudzanie\um0427\FWLib\library\src/stm32f10x_tim.c:2577
   2:	4770      	bx	lr
Disassembly of section .text.TIM_SetCompare1:

00000000 <TIM_SetCompare1>:
TIM_SetCompare1():
D:\STM32\Program\1.11_Odchudzanie\um0427\FWLib\library\src/stm32f10x_tim.c:2589
   0:	8681      	strh	r1, [r0, #52]
D:\STM32\Program\1.11_Odchudzanie\um0427\FWLib\library\src/stm32f10x_tim.c:2595
   2:	4770      	bx	lr
Disassembly of section .text.TIM_SetCompare2:

00000000 <TIM_SetCompare2>:
TIM_SetCompare2():
D:\STM32\Program\1.11_Odchudzanie\um0427\FWLib\library\src/stm32f10x_tim.c:2607
   0:	8701      	strh	r1, [r0, #56]
D:\STM32\Program\1.11_Odchudzanie\um0427\FWLib\library\src/stm32f10x_tim.c:2613
   2:	4770      	bx	lr
Disassembly of section .text.TIM_SetCompare3:

00000000 <TIM_SetCompare3>:
TIM_SetCompare3():
D:\STM32\Program\1.11_Odchudzanie\um0427\FWLib\library\src/stm32f10x_tim.c:2625
   0:	8781      	strh	r1, [r0, #60]
D:\STM32\Program\1.11_Odchudzanie\um0427\FWLib\library\src/stm32f10x_tim.c:2631
   2:	4770      	bx	lr
Disassembly of section .text.TIM_SetCompare4:

00000000 <TIM_SetCompare4>:
TIM_SetCompare4():
D:\STM32\Program\1.11_Odchudzanie\um0427\FWLib\library\src/stm32f10x_tim.c:2643
   0:	f8a0 1040 	strh.w	r1, [r0, #64]
D:\STM32\Program\1.11_Odchudzanie\um0427\FWLib\library\src/stm32f10x_tim.c:2649
   4:	4770      	bx	lr
   6:	46c0      	nop			(mov r8, r8)
Disassembly of section .text.TIM_SetIC1Prescaler:

00000000 <TIM_SetIC1Prescaler>:
TIM_SetIC1Prescaler():
D:\STM32\Program\1.11_Odchudzanie\um0427\FWLib\library\src/stm32f10x_tim.c:2667
   0:	8b03      	ldrh	r3, [r0, #24]
   2:	f023 030c 	bic.w	r3, r3, #12	; 0xc
   6:	041b      	lsls	r3, r3, #16
   8:	0c1b      	lsrs	r3, r3, #16
   a:	8303      	strh	r3, [r0, #24]
D:\STM32\Program\1.11_Odchudzanie\um0427\FWLib\library\src/stm32f10x_tim.c:2676
   c:	8b03      	ldrh	r3, [r0, #24]
   e:	b29b      	uxth	r3, r3
  10:	4319      	orrs	r1, r3
  12:	8301      	strh	r1, [r0, #24]
D:\STM32\Program\1.11_Odchudzanie\um0427\FWLib\library\src/stm32f10x_tim.c:2677
  14:	4770      	bx	lr
  16:	46c0      	nop			(mov r8, r8)
Disassembly of section .text.TIM_SetIC2Prescaler:

00000000 <TIM_SetIC2Prescaler>:
TIM_SetIC2Prescaler():
D:\STM32\Program\1.11_Odchudzanie\um0427\FWLib\library\src/stm32f10x_tim.c:2695
   0:	8b03      	ldrh	r3, [r0, #24]
   2:	f423 6340 	bic.w	r3, r3, #3072	; 0xc00
   6:	041b      	lsls	r3, r3, #16
   8:	0c1b      	lsrs	r3, r3, #16
   a:	8303      	strh	r3, [r0, #24]
D:\STM32\Program\1.11_Odchudzanie\um0427\FWLib\library\src/stm32f10x_tim.c:2704
   c:	8b03      	ldrh	r3, [r0, #24]
   e:	b29b      	uxth	r3, r3
  10:	ea43 2301 	orr.w	r3, r3, r1, lsl #8
  14:	b29b      	uxth	r3, r3
  16:	8303      	strh	r3, [r0, #24]
D:\STM32\Program\1.11_Odchudzanie\um0427\FWLib\library\src/stm32f10x_tim.c:2705
  18:	4770      	bx	lr
  1a:	46c0      	nop			(mov r8, r8)
Disassembly of section .text.TIM_SetIC3Prescaler:

00000000 <TIM_SetIC3Prescaler>:
TIM_SetIC3Prescaler():
D:\STM32\Program\1.11_Odchudzanie\um0427\FWLib\library\src/stm32f10x_tim.c:2723
   0:	8b83      	ldrh	r3, [r0, #28]
   2:	f023 030c 	bic.w	r3, r3, #12	; 0xc
   6:	041b      	lsls	r3, r3, #16
   8:	0c1b      	lsrs	r3, r3, #16
   a:	8383      	strh	r3, [r0, #28]
D:\STM32\Program\1.11_Odchudzanie\um0427\FWLib\library\src/stm32f10x_tim.c:2732
   c:	8b83      	ldrh	r3, [r0, #28]
   e:	b29b      	uxth	r3, r3
  10:	4319      	orrs	r1, r3
  12:	8381      	strh	r1, [r0, #28]
D:\STM32\Program\1.11_Odchudzanie\um0427\FWLib\library\src/stm32f10x_tim.c:2733
  14:	4770      	bx	lr
  16:	46c0      	nop			(mov r8, r8)
Disassembly of section .text.TIM_SetIC4Prescaler:

00000000 <TIM_SetIC4Prescaler>:
TIM_SetIC4Prescaler():
D:\STM32\Program\1.11_Odchudzanie\um0427\FWLib\library\src/stm32f10x_tim.c:2751
   0:	8b83      	ldrh	r3, [r0, #28]
   2:	f423 6340 	bic.w	r3, r3, #3072	; 0xc00
   6:	041b      	lsls	r3, r3, #16
   8:	0c1b      	lsrs	r3, r3, #16
   a:	8383      	strh	r3, [r0, #28]
D:\STM32\Program\1.11_Odchudzanie\um0427\FWLib\library\src/stm32f10x_tim.c:2760
   c:	8b83      	ldrh	r3, [r0, #28]
   e:	b29b      	uxth	r3, r3
  10:	ea43 2301 	orr.w	r3, r3, r1, lsl #8
  14:	b29b      	uxth	r3, r3
  16:	8383      	strh	r3, [r0, #28]
D:\STM32\Program\1.11_Odchudzanie\um0427\FWLib\library\src/stm32f10x_tim.c:2761
  18:	4770      	bx	lr
  1a:	46c0      	nop			(mov r8, r8)
Disassembly of section .text.TIM_SetClockDivision:

00000000 <TIM_SetClockDivision>:
TIM_SetClockDivision():
D:\STM32\Program\1.11_Odchudzanie\um0427\FWLib\library\src/stm32f10x_tim.c:2777
   0:	8803      	ldrh	r3, [r0, #0]
   2:	b2db      	uxtb	r3, r3
   4:	8003      	strh	r3, [r0, #0]
D:\STM32\Program\1.11_Odchudzanie\um0427\FWLib\library\src/stm32f10x_tim.c:2786
   6:	8803      	ldrh	r3, [r0, #0]
   8:	b29b      	uxth	r3, r3
   a:	4319      	orrs	r1, r3
   c:	8001      	strh	r1, [r0, #0]
D:\STM32\Program\1.11_Odchudzanie\um0427\FWLib\library\src/stm32f10x_tim.c:2787
   e:	4770      	bx	lr
Disassembly of section .text.TIM_GetCapture1:

00000000 <TIM_GetCapture1>:
TIM_GetCapture1():
D:\STM32\Program\1.11_Odchudzanie\um0427\FWLib\library\src/stm32f10x_tim.c:2797
   0:	8e80      	ldrh	r0, [r0, #52]
   2:	b280      	uxth	r0, r0
   4:	4770      	bx	lr
   6:	46c0      	nop			(mov r8, r8)
Disassembly of section .text.TIM_GetCapture2:

00000000 <TIM_GetCapture2>:
TIM_GetCapture2():
D:\STM32\Program\1.11_Odchudzanie\um0427\FWLib\library\src/stm32f10x_tim.c:2814
   0:	8f00      	ldrh	r0, [r0, #56]
   2:	b280      	uxth	r0, r0
   4:	4770      	bx	lr
   6:	46c0      	nop			(mov r8, r8)
Disassembly of section .text.TIM_GetCapture3:

00000000 <TIM_GetCapture3>:
TIM_GetCapture3():
D:\STM32\Program\1.11_Odchudzanie\um0427\FWLib\library\src/stm32f10x_tim.c:2831
   0:	8f80      	ldrh	r0, [r0, #60]
   2:	b280      	uxth	r0, r0
   4:	4770      	bx	lr
   6:	46c0      	nop			(mov r8, r8)
Disassembly of section .text.TIM_GetCapture4:

00000000 <TIM_GetCapture4>:
TIM_GetCapture4():
D:\STM32\Program\1.11_Odchudzanie\um0427\FWLib\library\src/stm32f10x_tim.c:2848
   0:	f8b0 0040 	ldrh.w	r0, [r0, #64]
   4:	b280      	uxth	r0, r0
   6:	4770      	bx	lr
Disassembly of section .text.TIM_GetCounter:

00000000 <TIM_GetCounter>:
TIM_GetCounter():
D:\STM32\Program\1.11_Odchudzanie\um0427\FWLib\library\src/stm32f10x_tim.c:2864
   0:	8c80      	ldrh	r0, [r0, #36]
   2:	b280      	uxth	r0, r0
   4:	4770      	bx	lr
   6:	46c0      	nop			(mov r8, r8)
Disassembly of section .text.TIM_GetPrescaler:

00000000 <TIM_GetPrescaler>:
TIM_GetPrescaler():
D:\STM32\Program\1.11_Odchudzanie\um0427\FWLib\library\src/stm32f10x_tim.c:2880
   0:	8d00      	ldrh	r0, [r0, #40]
   2:	b280      	uxth	r0, r0
   4:	4770      	bx	lr
   6:	46c0      	nop			(mov r8, r8)
Disassembly of section .text.TIM_GetFlagStatus:

00000000 <TIM_GetFlagStatus>:
TIM_GetFlagStatus():
D:\STM32\Program\1.11_Odchudzanie\um0427\FWLib\library\src/stm32f10x_tim.c:2910
   0:	8a03      	ldrh	r3, [r0, #16]
   2:	4219      	tst	r1, r3
D:\STM32\Program\1.11_Odchudzanie\um0427\FWLib\library\src/stm32f10x_tim.c:2927
   4:	bf0c      	ite	eq
   6:	2000      	moveq	r0, #0
   8:	2001      	movne	r0, #1
   a:	4770      	bx	lr
Disassembly of section .text.TIM_ClearFlag:

00000000 <TIM_ClearFlag>:
TIM_ClearFlag():
D:\STM32\Program\1.11_Odchudzanie\um0427\FWLib\library\src/stm32f10x_tim.c:2951
   0:	43c9      	mvns	r1, r1
   2:	b289      	uxth	r1, r1
   4:	8201      	strh	r1, [r0, #16]
D:\STM32\Program\1.11_Odchudzanie\um0427\FWLib\library\src/stm32f10x_tim.c:2958
   6:	4770      	bx	lr
Disassembly of section .text.TIM_GetITStatus:

00000000 <TIM_GetITStatus>:
TIM_GetITStatus():
D:\STM32\Program\1.11_Odchudzanie\um0427\FWLib\library\src/stm32f10x_tim.c:2979
   0:	8a02      	ldrh	r2, [r0, #16]
D:\STM32\Program\1.11_Odchudzanie\um0427\FWLib\library\src/stm32f10x_tim.c:2990
   2:	8983      	ldrh	r3, [r0, #12]
D:\STM32\Program\1.11_Odchudzanie\um0427\FWLib\library\src/stm32f10x_tim.c:2992
   4:	ea11 0002 	ands.w	r0, r1, r2
D:\STM32\Program\1.11_Odchudzanie\um0427\FWLib\library\src/stm32f10x_tim.c:2979
   8:	b29b      	uxth	r3, r3
D:\STM32\Program\1.11_Odchudzanie\um0427\FWLib\library\src/stm32f10x_tim.c:2992
   a:	d003      	beq.n	14 <TIM_GetITStatus+0x14>
   c:	4219      	tst	r1, r3
   e:	bf0c      	ite	eq
  10:	2000      	moveq	r0, #0
  12:	2001      	movne	r0, #1
D:\STM32\Program\1.11_Odchudzanie\um0427\FWLib\library\src/stm32f10x_tim.c:3001
  14:	4770      	bx	lr
  16:	46c0      	nop			(mov r8, r8)
Disassembly of section .text.TIM_ClearITPendingBit:

00000000 <TIM_ClearITPendingBit>:
TIM_ClearITPendingBit():
D:\STM32\Program\1.11_Odchudzanie\um0427\FWLib\library\src/stm32f10x_tim.c:3022
   0:	43c9      	mvns	r1, r1
   2:	b289      	uxth	r1, r1
   4:	8201      	strh	r1, [r0, #16]
D:\STM32\Program\1.11_Odchudzanie\um0427\FWLib\library\src/stm32f10x_tim.c:3029
   6:	4770      	bx	lr
Disassembly of section .text.TI1_Config:

00000000 <TI1_Config>:
TI1_Config():
D:\STM32\Program\1.11_Odchudzanie\um0427\FWLib\library\src/stm32f10x_tim.c:3055
   0:	b530      	push	{r4, r5, lr}
D:\STM32\Program\1.11_Odchudzanie\um0427\FWLib\library\src/stm32f10x_tim.c:3059
   2:	8c04      	ldrh	r4, [r0, #32]
   4:	f024 0401 	bic.w	r4, r4, #1	; 0x1
   8:	0424      	lsls	r4, r4, #16
   a:	0c24      	lsrs	r4, r4, #16
   c:	8404      	strh	r4, [r0, #32]
D:\STM32\Program\1.11_Odchudzanie\um0427\FWLib\library\src/stm32f10x_tim.c:3061
   e:	8b04      	ldrh	r4, [r0, #24]
D:\STM32\Program\1.11_Odchudzanie\um0427\FWLib\library\src/stm32f10x_tim.c:3062
  10:	8c05      	ldrh	r5, [r0, #32]
D:\STM32\Program\1.11_Odchudzanie\um0427\FWLib\library\src/stm32f10x_tim.c:3066
  12:	f024 04f3 	bic.w	r4, r4, #243	; 0xf3
  16:	0424      	lsls	r4, r4, #16
D:\STM32\Program\1.11_Odchudzanie\um0427\FWLib\library\src/stm32f10x_tim.c:3070
  18:	f025 0502 	bic.w	r5, r5, #2	; 0x2
D:\STM32\Program\1.11_Odchudzanie\um0427\FWLib\library\src/stm32f10x_tim.c:3066
  1c:	0c24      	lsrs	r4, r4, #16
D:\STM32\Program\1.11_Odchudzanie\um0427\FWLib\library\src/stm32f10x_tim.c:3070
  1e:	042d      	lsls	r5, r5, #16
D:\STM32\Program\1.11_Odchudzanie\um0427\FWLib\library\src/stm32f10x_tim.c:3066
  20:	4322      	orrs	r2, r4
D:\STM32\Program\1.11_Odchudzanie\um0427\FWLib\library\src/stm32f10x_tim.c:3070
  22:	0c2d      	lsrs	r5, r5, #16
D:\STM32\Program\1.11_Odchudzanie\um0427\FWLib\library\src/stm32f10x_tim.c:3066
  24:	ea42 1203 	orr.w	r2, r2, r3, lsl #4
D:\STM32\Program\1.11_Odchudzanie\um0427\FWLib\library\src/stm32f10x_tim.c:3070
  28:	f045 0501 	orr.w	r5, r5, #1	; 0x1
D:\STM32\Program\1.11_Odchudzanie\um0427\FWLib\library\src/stm32f10x_tim.c:3066
  2c:	b292      	uxth	r2, r2
D:\STM32\Program\1.11_Odchudzanie\um0427\FWLib\library\src/stm32f10x_tim.c:3070
  2e:	430d      	orrs	r5, r1
D:\STM32\Program\1.11_Odchudzanie\um0427\FWLib\library\src/stm32f10x_tim.c:3073
  30:	8302      	strh	r2, [r0, #24]
D:\STM32\Program\1.11_Odchudzanie\um0427\FWLib\library\src/stm32f10x_tim.c:3074
  32:	8405      	strh	r5, [r0, #32]
D:\STM32\Program\1.11_Odchudzanie\um0427\FWLib\library\src/stm32f10x_tim.c:3075
  34:	bd30      	pop	{r4, r5, pc}
  36:	46c0      	nop			(mov r8, r8)
Disassembly of section .text.TI2_Config:

00000000 <TI2_Config>:
TI2_Config():
D:\STM32\Program\1.11_Odchudzanie\um0427\FWLib\library\src/stm32f10x_tim.c:3101
   0:	b530      	push	{r4, r5, lr}
D:\STM32\Program\1.11_Odchudzanie\um0427\FWLib\library\src/stm32f10x_tim.c:3105
   2:	8c04      	ldrh	r4, [r0, #32]
   4:	f024 0410 	bic.w	r4, r4, #16	; 0x10
   8:	0424      	lsls	r4, r4, #16
   a:	0c24      	lsrs	r4, r4, #16
   c:	8404      	strh	r4, [r0, #32]
D:\STM32\Program\1.11_Odchudzanie\um0427\FWLib\library\src/stm32f10x_tim.c:3107
   e:	8b04      	ldrh	r4, [r0, #24]
D:\STM32\Program\1.11_Odchudzanie\um0427\FWLib\library\src/stm32f10x_tim.c:3108
  10:	8c05      	ldrh	r5, [r0, #32]
D:\STM32\Program\1.11_Odchudzanie\um0427\FWLib\library\src/stm32f10x_tim.c:3112
  12:	f424 7440 	bic.w	r4, r4, #768	; 0x300
  16:	0524      	lsls	r4, r4, #20
D:\STM32\Program\1.11_Odchudzanie\um0427\FWLib\library\src/stm32f10x_tim.c:3118
  18:	f025 0520 	bic.w	r5, r5, #32	; 0x20
D:\STM32\Program\1.11_Odchudzanie\um0427\FWLib\library\src/stm32f10x_tim.c:3112
  1c:	0d24      	lsrs	r4, r4, #20
D:\STM32\Program\1.11_Odchudzanie\um0427\FWLib\library\src/stm32f10x_tim.c:3118
  1e:	042d      	lsls	r5, r5, #16
D:\STM32\Program\1.11_Odchudzanie\um0427\FWLib\library\src/stm32f10x_tim.c:3113
  20:	ea44 2402 	orr.w	r4, r4, r2, lsl #8
D:\STM32\Program\1.11_Odchudzanie\um0427\FWLib\library\src/stm32f10x_tim.c:3118
  24:	0c2d      	lsrs	r5, r5, #16
D:\STM32\Program\1.11_Odchudzanie\um0427\FWLib\library\src/stm32f10x_tim.c:3113
  26:	b2a4      	uxth	r4, r4
D:\STM32\Program\1.11_Odchudzanie\um0427\FWLib\library\src/stm32f10x_tim.c:3118
  28:	f045 0510 	orr.w	r5, r5, #16	; 0x10
D:\STM32\Program\1.11_Odchudzanie\um0427\FWLib\library\src/stm32f10x_tim.c:3114
  2c:	ea44 3403 	orr.w	r4, r4, r3, lsl #12
D:\STM32\Program\1.11_Odchudzanie\um0427\FWLib\library\src/stm32f10x_tim.c:3118
  30:	ea45 1501 	orr.w	r5, r5, r1, lsl #4
D:\STM32\Program\1.11_Odchudzanie\um0427\FWLib\library\src/stm32f10x_tim.c:3114
  34:	b2a4      	uxth	r4, r4
D:\STM32\Program\1.11_Odchudzanie\um0427\FWLib\library\src/stm32f10x_tim.c:3118
  36:	b2ad      	uxth	r5, r5
D:\STM32\Program\1.11_Odchudzanie\um0427\FWLib\library\src/stm32f10x_tim.c:3121
  38:	8304      	strh	r4, [r0, #24]
D:\STM32\Program\1.11_Odchudzanie\um0427\FWLib\library\src/stm32f10x_tim.c:3122
  3a:	8405      	strh	r5, [r0, #32]
D:\STM32\Program\1.11_Odchudzanie\um0427\FWLib\library\src/stm32f10x_tim.c:3123
  3c:	bd30      	pop	{r4, r5, pc}
  3e:	46c0      	nop			(mov r8, r8)
Disassembly of section .text.TIM_TIxExternalClockConfig:

00000000 <TIM_TIxExternalClockConfig>:
TIM_TIxExternalClockConfig():
D:\STM32\Program\1.11_Odchudzanie\um0427\FWLib\library\src/stm32f10x_tim.c:1071
   0:	b570      	push	{r4, r5, r6, lr}
   2:	460d      	mov	r5, r1
D:\STM32\Program\1.11_Odchudzanie\um0427\FWLib\library\src/stm32f10x_tim.c:1079
   4:	2d60      	cmp	r5, #96
D:\STM32\Program\1.11_Odchudzanie\um0427\FWLib\library\src/stm32f10x_tim.c:1071
   6:	4604      	mov	r4, r0
   8:	4611      	mov	r1, r2
D:\STM32\Program\1.11_Odchudzanie\um0427\FWLib\library\src/stm32f10x_tim.c:1079
   a:	d103      	bne.n	14 <TIM_TIxExternalClockConfig+0x14>
D:\STM32\Program\1.11_Odchudzanie\um0427\FWLib\library\src/stm32f10x_tim.c:1081
   c:	2201      	movs	r2, #1
   e:	f7ff fffe 	bl	0 <TIM_TIxExternalClockConfig>
  12:	e002      	b.n	1a <TIM_TIxExternalClockConfig+0x1a>
D:\STM32\Program\1.11_Odchudzanie\um0427\FWLib\library\src/stm32f10x_tim.c:1085
  14:	2201      	movs	r2, #1
  16:	f7ff fffe 	bl	0 <TIM_TIxExternalClockConfig>
D:\STM32\Program\1.11_Odchudzanie\um0427\FWLib\library\src/stm32f10x_tim.c:1089
  1a:	4620      	mov	r0, r4
  1c:	4629      	mov	r1, r5
  1e:	f7ff fffe 	bl	0 <TIM_TIxExternalClockConfig>
D:\STM32\Program\1.11_Odchudzanie\um0427\FWLib\library\src/stm32f10x_tim.c:1092
  22:	8923      	ldrh	r3, [r4, #8]
  24:	b29b      	uxth	r3, r3
  26:	f043 0307 	orr.w	r3, r3, #7	; 0x7
  2a:	8123      	strh	r3, [r4, #8]
D:\STM32\Program\1.11_Odchudzanie\um0427\FWLib\library\src/stm32f10x_tim.c:1093
  2c:	bd70      	pop	{r4, r5, r6, pc}
  2e:	46c0      	nop			(mov r8, r8)
Disassembly of section .text.TIM_PWMIConfig:

00000000 <TIM_PWMIConfig>:
TIM_PWMIConfig():
D:\STM32\Program\1.11_Odchudzanie\um0427\FWLib\library\src/stm32f10x_tim.c:651
   0:	e92d 41f0 	stmdb	sp!, {r4, r5, r6, r7, r8, lr}
   4:	460c      	mov	r4, r1
D:\STM32\Program\1.11_Odchudzanie\um0427\FWLib\library\src/stm32f10x_tim.c:669
   6:	88a2      	ldrh	r2, [r4, #4]
D:\STM32\Program\1.11_Odchudzanie\um0427\FWLib\library\src/stm32f10x_tim.c:659
   8:	8849      	ldrh	r1, [r1, #2]
D:\STM32\Program\1.11_Odchudzanie\um0427\FWLib\library\src/stm32f10x_tim.c:678
   a:	8823      	ldrh	r3, [r4, #0]
D:\STM32\Program\1.11_Odchudzanie\um0427\FWLib\library\src/stm32f10x_tim.c:651
   c:	4605      	mov	r5, r0
D:\STM32\Program\1.11_Odchudzanie\um0427\FWLib\library\src/stm32f10x_tim.c:659
   e:	2900      	cmp	r1, #0
  10:	bf0c      	ite	eq
  12:	2702      	moveq	r7, #2
  14:	2700      	movne	r7, #0
D:\STM32\Program\1.11_Odchudzanie\um0427\FWLib\library\src/stm32f10x_tim.c:669
  16:	2a01      	cmp	r2, #1
  18:	bf14      	ite	ne
  1a:	2601      	movne	r6, #1
  1c:	2602      	moveq	r6, #2
  1e:	f8b4 e008 	ldrh.w	lr, [r4, #8]
D:\STM32\Program\1.11_Odchudzanie\um0427\FWLib\library\src/stm32f10x_tim.c:678
  22:	b98b      	cbnz	r3, 48 <TIM_PWMIConfig+0x48>
D:\STM32\Program\1.11_Odchudzanie\um0427\FWLib\library\src/stm32f10x_tim.c:681
  24:	4673      	mov	r3, lr
  26:	f7ff fffe 	bl	0 <TIM_PWMIConfig>
D:\STM32\Program\1.11_Odchudzanie\um0427\FWLib\library\src/stm32f10x_tim.c:685
  2a:	4628      	mov	r0, r5
  2c:	88e1      	ldrh	r1, [r4, #6]
  2e:	f7ff fffe 	bl	0 <TIM_PWMIConfig>
D:\STM32\Program\1.11_Odchudzanie\um0427\FWLib\library\src/stm32f10x_tim.c:688
  32:	4628      	mov	r0, r5
  34:	4639      	mov	r1, r7
  36:	4632      	mov	r2, r6
  38:	8923      	ldrh	r3, [r4, #8]
  3a:	f7ff fffe 	bl	0 <TIM_PWMIConfig>
D:\STM32\Program\1.11_Odchudzanie\um0427\FWLib\library\src/stm32f10x_tim.c:691
  3e:	4628      	mov	r0, r5
  40:	88e1      	ldrh	r1, [r4, #6]
  42:	f7ff fffe 	bl	0 <TIM_PWMIConfig>
  46:	e010      	b.n	6a <TIM_PWMIConfig+0x6a>
D:\STM32\Program\1.11_Odchudzanie\um0427\FWLib\library\src/stm32f10x_tim.c:696
  48:	4673      	mov	r3, lr
  4a:	f7ff fffe 	bl	0 <TIM_PWMIConfig>
D:\STM32\Program\1.11_Odchudzanie\um0427\FWLib\library\src/stm32f10x_tim.c:700
  4e:	4628      	mov	r0, r5
  50:	88e1      	ldrh	r1, [r4, #6]
  52:	f7ff fffe 	bl	0 <TIM_PWMIConfig>
D:\STM32\Program\1.11_Odchudzanie\um0427\FWLib\library\src/stm32f10x_tim.c:703
  56:	4628      	mov	r0, r5
  58:	4639      	mov	r1, r7
  5a:	4632      	mov	r2, r6
  5c:	8923      	ldrh	r3, [r4, #8]
  5e:	f7ff fffe 	bl	0 <TIM_PWMIConfig>
D:\STM32\Program\1.11_Odchudzanie\um0427\FWLib\library\src/stm32f10x_tim.c:706
  62:	4628      	mov	r0, r5
  64:	88e1      	ldrh	r1, [r4, #6]
  66:	f7ff fffe 	bl	0 <TIM_PWMIConfig>
D:\STM32\Program\1.11_Odchudzanie\um0427\FWLib\library\src/stm32f10x_tim.c:708
  6a:	e8bd 81f0 	ldmia.w	sp!, {r4, r5, r6, r7, r8, pc}
  6e:	46c0      	nop			(mov r8, r8)
Disassembly of section .text.TIM_ICInit:

00000000 <TIM_ICInit>:
TIM_ICInit():
D:\STM32\Program\1.11_Odchudzanie\um0427\FWLib\library\src/stm32f10x_tim.c:586
   0:	880b      	ldrh	r3, [r1, #0]
   2:	b570      	push	{r4, r5, r6, lr}
   4:	4604      	mov	r4, r0
   6:	460d      	mov	r5, r1
D:\STM32\Program\1.11_Odchudzanie\um0427\FWLib\library\src/stm32f10x_tim.c:595
   8:	b94b      	cbnz	r3, 1e <TIM_ICInit+0x1e>
D:\STM32\Program\1.11_Odchudzanie\um0427\FWLib\library\src/stm32f10x_tim.c:598
   a:	8849      	ldrh	r1, [r1, #2]
   c:	88aa      	ldrh	r2, [r5, #4]
   e:	892b      	ldrh	r3, [r5, #8]
  10:	f7ff fffe 	bl	0 <TIM_ICInit>
D:\STM32\Program\1.11_Odchudzanie\um0427\FWLib\library\src/stm32f10x_tim.c:603
  14:	4620      	mov	r0, r4
  16:	88e9      	ldrh	r1, [r5, #6]
  18:	f7ff fffe 	bl	0 <TIM_ICInit>
  1c:	e052      	b.n	c4 <TIM_ICInit+0xc4>
D:\STM32\Program\1.11_Odchudzanie\um0427\FWLib\library\src/stm32f10x_tim.c:605
  1e:	2b04      	cmp	r3, #4
  20:	d109      	bne.n	36 <TIM_ICInit+0x36>
D:\STM32\Program\1.11_Odchudzanie\um0427\FWLib\library\src/stm32f10x_tim.c:608
  22:	8849      	ldrh	r1, [r1, #2]
  24:	88aa      	ldrh	r2, [r5, #4]
  26:	892b      	ldrh	r3, [r5, #8]
  28:	f7ff fffe 	bl	0 <TIM_ICInit>
D:\STM32\Program\1.11_Odchudzanie\um0427\FWLib\library\src/stm32f10x_tim.c:613
  2c:	4620      	mov	r0, r4
  2e:	88e9      	ldrh	r1, [r5, #6]
  30:	f7ff fffe 	bl	0 <TIM_ICInit>
  34:	e046      	b.n	c4 <TIM_ICInit+0xc4>
D:\STM32\Program\1.11_Odchudzanie\um0427\FWLib\library\src/stm32f10x_tim.c:615
  36:	2b08      	cmp	r3, #8
  38:	f8b1 c002 	ldrh.w	ip, [r1, #2]
  3c:	f8b1 e004 	ldrh.w	lr, [r1, #4]
  40:	8909      	ldrh	r1, [r1, #8]
  42:	d11f      	bne.n	84 <TIM_ICInit+0x84>
TI3_Config():
D:\STM32\Program\1.11_Odchudzanie\um0427\FWLib\library\src/stm32f10x_tim.c:3153
  44:	8c03      	ldrh	r3, [r0, #32]
  46:	f423 7380 	bic.w	r3, r3, #256	; 0x100
  4a:	041b      	lsls	r3, r3, #16
  4c:	0c1b      	lsrs	r3, r3, #16
  4e:	8403      	strh	r3, [r0, #32]
D:\STM32\Program\1.11_Odchudzanie\um0427\FWLib\library\src/stm32f10x_tim.c:3155
  50:	8b83      	ldrh	r3, [r0, #28]
D:\STM32\Program\1.11_Odchudzanie\um0427\FWLib\library\src/stm32f10x_tim.c:3156
  52:	8c02      	ldrh	r2, [r0, #32]
D:\STM32\Program\1.11_Odchudzanie\um0427\FWLib\library\src/stm32f10x_tim.c:3161
  54:	f023 03f3 	bic.w	r3, r3, #243	; 0xf3
D:\STM32\Program\1.11_Odchudzanie\um0427\FWLib\library\src/stm32f10x_tim.c:3165
  58:	f422 7200 	bic.w	r2, r2, #512	; 0x200
D:\STM32\Program\1.11_Odchudzanie\um0427\FWLib\library\src/stm32f10x_tim.c:3161
  5c:	041b      	lsls	r3, r3, #16
D:\STM32\Program\1.11_Odchudzanie\um0427\FWLib\library\src/stm32f10x_tim.c:3165
  5e:	0412      	lsls	r2, r2, #16
D:\STM32\Program\1.11_Odchudzanie\um0427\FWLib\library\src/stm32f10x_tim.c:3161
  60:	0c1b      	lsrs	r3, r3, #16
D:\STM32\Program\1.11_Odchudzanie\um0427\FWLib\library\src/stm32f10x_tim.c:3165
  62:	0c12      	lsrs	r2, r2, #16
D:\STM32\Program\1.11_Odchudzanie\um0427\FWLib\library\src/stm32f10x_tim.c:3161
  64:	ea43 1301 	orr.w	r3, r3, r1, lsl #4
D:\STM32\Program\1.11_Odchudzanie\um0427\FWLib\library\src/stm32f10x_tim.c:3165
  68:	ea42 220c 	orr.w	r2, r2, ip, lsl #8
D:\STM32\Program\1.11_Odchudzanie\um0427\FWLib\library\src/stm32f10x_tim.c:3161
  6c:	b29b      	uxth	r3, r3
D:\STM32\Program\1.11_Odchudzanie\um0427\FWLib\library\src/stm32f10x_tim.c:3165
  6e:	b292      	uxth	r2, r2
D:\STM32\Program\1.11_Odchudzanie\um0427\FWLib\library\src/stm32f10x_tim.c:3161
  70:	ea43 030e 	orr.w	r3, r3, lr
D:\STM32\Program\1.11_Odchudzanie\um0427\FWLib\library\src/stm32f10x_tim.c:3165
  74:	f442 7280 	orr.w	r2, r2, #256	; 0x100
D:\STM32\Program\1.11_Odchudzanie\um0427\FWLib\library\src/stm32f10x_tim.c:3168
  78:	8383      	strh	r3, [r0, #28]
D:\STM32\Program\1.11_Odchudzanie\um0427\FWLib\library\src/stm32f10x_tim.c:3169
  7a:	8402      	strh	r2, [r0, #32]
TIM_ICInit():
D:\STM32\Program\1.11_Odchudzanie\um0427\FWLib\library\src/stm32f10x_tim.c:623
  7c:	88e9      	ldrh	r1, [r5, #6]
  7e:	f7ff fffe 	bl	0 <TIM_ICInit>
  82:	e01f      	b.n	c4 <TIM_ICInit+0xc4>
TI4_Config():
D:\STM32\Program\1.11_Odchudzanie\um0427\FWLib\library\src/stm32f10x_tim.c:3200
  84:	8c03      	ldrh	r3, [r0, #32]
  86:	f423 5380 	bic.w	r3, r3, #4096	; 0x1000
  8a:	041b      	lsls	r3, r3, #16
  8c:	0c1b      	lsrs	r3, r3, #16
  8e:	8403      	strh	r3, [r0, #32]
D:\STM32\Program\1.11_Odchudzanie\um0427\FWLib\library\src/stm32f10x_tim.c:3202
  90:	8b83      	ldrh	r3, [r0, #28]
D:\STM32\Program\1.11_Odchudzanie\um0427\FWLib\library\src/stm32f10x_tim.c:3203
  92:	8c02      	ldrh	r2, [r0, #32]
D:\STM32\Program\1.11_Odchudzanie\um0427\FWLib\library\src/stm32f10x_tim.c:3208
  94:	f423 7340 	bic.w	r3, r3, #768	; 0x300
  98:	051b      	lsls	r3, r3, #20
D:\STM32\Program\1.11_Odchudzanie\um0427\FWLib\library\src/stm32f10x_tim.c:3212
  9a:	f422 5200 	bic.w	r2, r2, #8192	; 0x2000
D:\STM32\Program\1.11_Odchudzanie\um0427\FWLib\library\src/stm32f10x_tim.c:3208
  9e:	0d1b      	lsrs	r3, r3, #20
D:\STM32\Program\1.11_Odchudzanie\um0427\FWLib\library\src/stm32f10x_tim.c:3212
  a0:	0412      	lsls	r2, r2, #16
D:\STM32\Program\1.11_Odchudzanie\um0427\FWLib\library\src/stm32f10x_tim.c:3208
  a2:	ea43 230e 	orr.w	r3, r3, lr, lsl #8
D:\STM32\Program\1.11_Odchudzanie\um0427\FWLib\library\src/stm32f10x_tim.c:3212
  a6:	0c12      	lsrs	r2, r2, #16
D:\STM32\Program\1.11_Odchudzanie\um0427\FWLib\library\src/stm32f10x_tim.c:3208
  a8:	b29b      	uxth	r3, r3
D:\STM32\Program\1.11_Odchudzanie\um0427\FWLib\library\src/stm32f10x_tim.c:3212
  aa:	ea42 320c 	orr.w	r2, r2, ip, lsl #12
D:\STM32\Program\1.11_Odchudzanie\um0427\FWLib\library\src/stm32f10x_tim.c:3208
  ae:	ea43 3301 	orr.w	r3, r3, r1, lsl #12
D:\STM32\Program\1.11_Odchudzanie\um0427\FWLib\library\src/stm32f10x_tim.c:3212
  b2:	b292      	uxth	r2, r2
D:\STM32\Program\1.11_Odchudzanie\um0427\FWLib\library\src/stm32f10x_tim.c:3208
  b4:	b29b      	uxth	r3, r3
D:\STM32\Program\1.11_Odchudzanie\um0427\FWLib\library\src/stm32f10x_tim.c:3212
  b6:	f442 5280 	orr.w	r2, r2, #4096	; 0x1000
D:\STM32\Program\1.11_Odchudzanie\um0427\FWLib\library\src/stm32f10x_tim.c:3215
  ba:	8383      	strh	r3, [r0, #28]
D:\STM32\Program\1.11_Odchudzanie\um0427\FWLib\library\src/stm32f10x_tim.c:3216
  bc:	8402      	strh	r2, [r0, #32]
TIM_ICInit():
D:\STM32\Program\1.11_Odchudzanie\um0427\FWLib\library\src/stm32f10x_tim.c:633
  be:	88e9      	ldrh	r1, [r5, #6]
  c0:	f7ff fffe 	bl	0 <TIM_ICInit>
D:\STM32\Program\1.11_Odchudzanie\um0427\FWLib\library\src/stm32f10x_tim.c:635
  c4:	bd70      	pop	{r4, r5, r6, pc}
  c6:	46c0      	nop			(mov r8, r8)
Disassembly of section .text.TIM_DeInit:

00000000 <TIM_DeInit>:
TIM_DeInit():
D:\STM32\Program\1.11_Odchudzanie\um0427\FWLib\library\src/stm32f10x_tim.c:135
   0:	b507      	push	{r0, r1, r2, lr}
D:\STM32\Program\1.11_Odchudzanie\um0427\FWLib\library\src/stm32f10x_tim.c:139
   2:	4b2e      	ldr	r3, [pc, #184]	(bc <TIM_DeInit+0xbc>)
D:\STM32\Program\1.11_Odchudzanie\um0427\FWLib\library\src/stm32f10x_tim.c:135
   4:	9001      	str	r0, [sp, #4]
D:\STM32\Program\1.11_Odchudzanie\um0427\FWLib\library\src/stm32f10x_tim.c:139
   6:	4298      	cmp	r0, r3
   8:	d037      	beq.n	7a <TIM_DeInit+0x7a>
   a:	d80b      	bhi.n	24 <TIM_DeInit+0x24>
   c:	f5a3 6300 	sub.w	r3, r3, #2048	; 0x800
  10:	4298      	cmp	r0, r3
  12:	d026      	beq.n	62 <TIM_DeInit+0x62>
  14:	f503 6380 	add.w	r3, r3, #1024	; 0x400
  18:	4298      	cmp	r0, r3
  1a:	d028      	beq.n	6e <TIM_DeInit+0x6e>
  1c:	f1b0 4f80 	cmp.w	r0, #1073741824	; 0x40000000
  20:	d019      	beq.n	56 <TIM_DeInit+0x56>
  22:	e049      	b.n	b8 <TIM_DeInit+0xb8>
  24:	4b26      	ldr	r3, [pc, #152]	(c0 <TIM_DeInit+0xc0>)
  26:	4298      	cmp	r0, r3
  28:	d033      	beq.n	92 <TIM_DeInit+0x92>
  2a:	d804      	bhi.n	36 <TIM_DeInit+0x36>
  2c:	f5a3 6380 	sub.w	r3, r3, #1024	; 0x400
  30:	4298      	cmp	r0, r3
  32:	d028      	beq.n	86 <TIM_DeInit+0x86>
  34:	e040      	b.n	b8 <TIM_DeInit+0xb8>
  36:	4b23      	ldr	r3, [pc, #140]	(c4 <TIM_DeInit+0xc4>)
  38:	4298      	cmp	r0, r3
  3a:	d004      	beq.n	46 <TIM_DeInit+0x46>
  3c:	f503 6300 	add.w	r3, r3, #2048	; 0x800
  40:	4298      	cmp	r0, r3
  42:	d02f      	beq.n	a4 <TIM_DeInit+0xa4>
  44:	e038      	b.n	b8 <TIM_DeInit+0xb8>
D:\STM32\Program\1.11_Odchudzanie\um0427\FWLib\library\src/stm32f10x_tim.c:142
  46:	f44f 6000 	mov.w	r0, #2048	; 0x800
  4a:	2101      	movs	r1, #1
  4c:	f7ff fffe 	bl	0 <RCC_APB2PeriphResetCmd>
D:\STM32\Program\1.11_Odchudzanie\um0427\FWLib\library\src/stm32f10x_tim.c:143
  50:	f44f 6000 	mov.w	r0, #2048	; 0x800
  54:	e02d      	b.n	b2 <TIM_DeInit+0xb2>
D:\STM32\Program\1.11_Odchudzanie\um0427\FWLib\library\src/stm32f10x_tim.c:147
  56:	2001      	movs	r0, #1
  58:	4601      	mov	r1, r0
  5a:	f7ff fffe 	bl	0 <RCC_APB1PeriphResetCmd>
D:\STM32\Program\1.11_Odchudzanie\um0427\FWLib\library\src/stm32f10x_tim.c:148
  5e:	2001      	movs	r0, #1
  60:	e01c      	b.n	9c <TIM_DeInit+0x9c>
D:\STM32\Program\1.11_Odchudzanie\um0427\FWLib\library\src/stm32f10x_tim.c:152
  62:	2002      	movs	r0, #2
  64:	2101      	movs	r1, #1
  66:	f7ff fffe 	bl	0 <RCC_APB1PeriphResetCmd>
D:\STM32\Program\1.11_Odchudzanie\um0427\FWLib\library\src/stm32f10x_tim.c:153
  6a:	2002      	movs	r0, #2
  6c:	e016      	b.n	9c <TIM_DeInit+0x9c>
D:\STM32\Program\1.11_Odchudzanie\um0427\FWLib\library\src/stm32f10x_tim.c:157
  6e:	2004      	movs	r0, #4
  70:	2101      	movs	r1, #1
  72:	f7ff fffe 	bl	0 <RCC_APB1PeriphResetCmd>
D:\STM32\Program\1.11_Odchudzanie\um0427\FWLib\library\src/stm32f10x_tim.c:158
  76:	2004      	movs	r0, #4
  78:	e010      	b.n	9c <TIM_DeInit+0x9c>
D:\STM32\Program\1.11_Odchudzanie\um0427\FWLib\library\src/stm32f10x_tim.c:162
  7a:	2008      	movs	r0, #8
  7c:	2101      	movs	r1, #1
  7e:	f7ff fffe 	bl	0 <RCC_APB1PeriphResetCmd>
D:\STM32\Program\1.11_Odchudzanie\um0427\FWLib\library\src/stm32f10x_tim.c:163
  82:	2008      	movs	r0, #8
  84:	e00a      	b.n	9c <TIM_DeInit+0x9c>
D:\STM32\Program\1.11_Odchudzanie\um0427\FWLib\library\src/stm32f10x_tim.c:167
  86:	2010      	movs	r0, #16
  88:	2101      	movs	r1, #1
  8a:	f7ff fffe 	bl	0 <RCC_APB1PeriphResetCmd>
D:\STM32\Program\1.11_Odchudzanie\um0427\FWLib\library\src/stm32f10x_tim.c:168
  8e:	2010      	movs	r0, #16
  90:	e004      	b.n	9c <TIM_DeInit+0x9c>
D:\STM32\Program\1.11_Odchudzanie\um0427\FWLib\library\src/stm32f10x_tim.c:172
  92:	2020      	movs	r0, #32
  94:	2101      	movs	r1, #1
  96:	f7ff fffe 	bl	0 <RCC_APB1PeriphResetCmd>
D:\STM32\Program\1.11_Odchudzanie\um0427\FWLib\library\src/stm32f10x_tim.c:173
  9a:	2020      	movs	r0, #32
  9c:	2100      	movs	r1, #0
  9e:	f7ff fffe 	bl	0 <RCC_APB1PeriphResetCmd>
D:\STM32\Program\1.11_Odchudzanie\um0427\FWLib\library\src/stm32f10x_tim.c:174
  a2:	e009      	b.n	b8 <TIM_DeInit+0xb8>
D:\STM32\Program\1.11_Odchudzanie\um0427\FWLib\library\src/stm32f10x_tim.c:177
  a4:	f44f 5000 	mov.w	r0, #8192	; 0x2000
  a8:	2101      	movs	r1, #1
  aa:	f7ff fffe 	bl	0 <RCC_APB2PeriphResetCmd>
D:\STM32\Program\1.11_Odchudzanie\um0427\FWLib\library\src/stm32f10x_tim.c:178
  ae:	f44f 5000 	mov.w	r0, #8192	; 0x2000
  b2:	2100      	movs	r1, #0
  b4:	f7ff fffe 	bl	0 <RCC_APB2PeriphResetCmd>
D:\STM32\Program\1.11_Odchudzanie\um0427\FWLib\library\src/stm32f10x_tim.c:184
  b8:	bd0e      	pop	{r1, r2, r3, pc}
  ba:	46c0      	nop			(mov r8, r8)
  bc:	40000c00 	.word	0x40000c00
  c0:	40001400 	.word	0x40001400
  c4:	40012c00 	.word	0x40012c00
